:020000040800F2
:10000000D8100020050100080B380008E52800087A
:1000100009380008350F0008BD6000080000000026
:10002000000000000000000000000000FD46000885
:10003000B71A0008000000007D3D0008E5490008EF
:100040001F010008793B00081F0100081F0100087C
:100050001F0100081F0100081F0100081F01000800
:100060001F0100081F0100081F0100081F010008F0
:100070001F0100081F010008791500081F01000872
:100080001F0100081F010008410700081F010008A8
:100090001F0100081F0100081F0100081F010008C0
:1000A000554A0008354B00081F0100081F010008D1
:1000B000394B0008294E0008855000081F01000830
:1000C0001F0100081F0100081F0100081F01000890
:1000D0001F010008B55B00081F0100081F01000890
:1000E0001F0100081F0100081F010008DFF810D0E1
:1000F00000F0E8FA00480047FD710008AFF3008007
:10010000D81000200648804706480047FEE7FEE773
:10011000FEE7FEE7FEE7FEE7FEE7FEE7FEE7FEE7B7
:10012000054A0008ED0000082DE9F0410024061BF7
:10013000254671F1000605DA01240027D0EB0700FF
:1001400067EB0101161E73F1000605DA0027D2EBFA
:100150000702012567EB030300F0D0F986460E463F
:1001600017469C46AC4204D00025D0EB050E65EB4B
:10017000010624B10020D2EB000760EB030C7046AF
:1001800031463A466346BDE8F08140EA01039B07E9
:1001900003D009E008C9121F08C0042AFAD203E0FC
:1001A00011F8013B00F8013B521EF9D2704780EA7A
:1001B000010210B502F00043400022D04A001FD0D7
:1001C000010E01EB1261C0F35600C2F3560240F477
:1001D000000042F40002A0FB022000047F39140456
:1001E00000D0401C50EA124001D44000491EC2B267
:1001F0000C0604EBD010401C4008802A02D003E01B
:10020000002010BD20F00100002900DA0020184372
:1002100010BD2DE9FE4F81EA030404F0004421F0F3
:10022000004100944FF0000B23F0004350EA01041A
:100230005ED052EA03045BD0C3F30A54C1F30A55FB
:100240002C44A4F2F3340194A0FB0254C1F3130133
:1002500041F48011C3F3130343F4801301FB024400
:1002600000FB034E840A970A44EA815447EA835705
:10027000A4FB076802958D0A05FB07854FEA932CBE
:1002800004FB0C542705029D4FEA065847EA16372F
:10029000B5EB08056EEB070C870E920E47EA811747
:1002A00042EA8312A7FB0201B6EB0B0164EB0004E8
:1002B0002B0D43EA0C335E1844EB1C50DA465146D2
:1002C000E7FB0201C5F313044FEA0B3343EA14536F
:1002D0004FEA0432019C43EA0603A4F10C040294A1
:1002E000009CCDE900B400F09FF903B0BDE8F08FA9
:1002F00000200146F9E72DE9F04D81EA030404F0FE
:10030000004B21F0004514464FF0000A23F0004155
:1003100050EA050220D054EA01021DD0C5F30A5765
:100320000246C5F31303C1F31300C1F30A5640F4A8
:10033000801543F48013A7EB0608101BD64608F27D
:10034000FD3873EB050002D308F1010801E09218B3
:100350005B41B8F1000F03DA00200146BDE8F08DE3
:1003600000204FF48011064684460EE0171B73EB05
:10037000050705D3121B63EB050306434CEA010C8A
:1003800049084FEA300092185B4150EA0107EDD16D
:1003900052EA030012D082EA040083EA050108430E
:1003A00005D0101BAB4106D20122002306E000223B
:1003B0004FF0004302E06FF0010253101AEB060009
:1003C0004CEB085110EB0A0041EB0B01BDE8F04D7E
:1003D00000F01BB970B521F0004303430CD0C1F30A
:1003E0000A550024D5EB040564EB0403D617AD1AB7
:1003F000B34102DB0020014670BD201841EB0251E1
:1004000070BDC10F80EAE0700844CA07962300213E
:1004100000F0CDB896230022114600F0C8B80EB502
:10042000C10F80EAE0700844CA07002140F233435C
:100430008DE80E000A460B4600F0F6F803B000BD4A
:100440000EB540F2334102910021CDE900110A4678
:100450000B4600F0E9F803B000BD00F0004220F0C8
:100460000040C10DC0F3160040F400007F2901DAFE
:1004700000207047962903DCC1F19601C84001E0D5
:1004800096398840002AF4D04042704770B5C1F3D5
:100490000A5201F000450024C1F3130140F2FF337A
:1004A00041F480119A4201DA002070BD40F23343DA
:1004B0009A42A2F2334203DC524200F05FF800E0BD
:1004C00090402C43F1D0404270BDC1F30A5210B5A8
:1004D000C1F3130140F2FF3341F480119A4201DA73
:1004E000002010BD40F233439A42A2F2334203DCB3
:1004F000524200F043F810BD904010BD2DE9F05F6E
:100500000546002092469B46884606468146402482
:100510001BE0284641464746224600F02FF8534646
:100520005A46C01A914110D311461846224600F08F
:1005300016F82D1A67EB01084F46224601200021CC
:1005400000F00DF817EB00094E41201EA4F1010444
:10055000DFDC484631462A464346BDE8F09F202A64
:1005600004DB203A00FA02F1002070479140C2F10A
:10057000200320FA03F3194390407047202A04DB3C
:10058000203A21FA02F00021704721FA02F3D0400C
:10059000C2F1200291400843194670470029A8BFC4
:1005A0007047401C490008BF20F00100704710B49C
:1005B000B0FA80FC00FA0CF050EA010404BF10BC51
:1005C000704749B1CCF1200421FA04F411FA0CF17E
:1005D00018BF012121430843A3EB0C01CB1D4FEAB7
:1005E00000614FEA102042BF002010BC704700EBB2
:1005F000C35010440029A4BF10BC7047401C4900E0
:1006000008BF20F0010010BC704710B5141E73F134
:10061000000408DA401C41F1000192185B411A43C2
:1006200001D120F0010010BD2DE9F04D92469B460E
:1006300011B1B1FA81F202E0B0FA80F220329046B4
:10064000FFF78DFF04460F4640EA0A0041EA0B011E
:1006500053465A46084313D0114653EA010019D0B5
:10066000C8F140025046FFF789FF05460E46504646
:1006700059464246FFF773FF084305D0012004E0C6
:1006800020463946BDE8F08D0020054346EAE07675
:100690002C4337430A986305E40AA0EB08000022C4
:1006A000FD0A44EA47540A3002D500200146E9E732
:1006B000010510196941DDE9084500196941BDE8E6
:1006C000F04DA2E7064C074D06E0E06840F001035C
:1006D00094E8070098471034AC42F6D3FFF70AFDC0
:1006E000409500086095000870B58C1810F8015B03
:1006F00015F0070301D110F8013B2A1106D110F8BB
:10070000012B03E010F8016B01F8016B5B1EF9D1BE
:100710002B0705D40023521E0DD401F8013BFAE744
:1007200010F8013BCB1A921C03E013F8015B01F8AF
:10073000015B521EF9D5A142D8D3002070BD000044
:1007400070B54E4C4FF490652946204600F019FADA
:10075000002864D02946204600F0A6F848490888B9
:10076000401C08800121204600F0EAFA454942F287
:100770001072B1F85000904202D2401CA1F8500013
:1007800006F018FF404DB5F91410B5F9120005F048
:10079000D7FD3E4CA5F84E002080A1682046884732
:1007A000A088A5F8500003F099F807F005F8384E36
:1007B000384C3078082833D045F6AC30606042F6CB
:1007C000EF60A06042F2C400E0603348008A2080FD
:1007D000208E6080A16B2F488847208E69882F4C1F
:1007E00008444FF6FF7101EA80006886207A4FF0D6
:1007F000000540071DD501F0EDFA294949F6A24050
:100800000880284840F21A62C188491C89B2C18018
:10081000914204D3A16821F00401A160C58070BD9C
:1008200041F2130060604FF48060A06040F61B50FE
:10083000CAE730780A281BD2DFE800F01A0616054E
:100840000A050D1A1114EAE7BDE8704005F01CBF57
:1008500007F08CFF08E0BDE8704002F089BD06F0AB
:10086000A5FA01E007F000F9BDE8704007F0FCB818
:1008700000F0F8FB84F8B65070BD00000024014081
:100880000007002044010020680000201C07002011
:10089000F7060020D8000020F4010020A00200206C
:1008A000442C0140200900206FEA112101607047AB
:1008B0000029816802D041F0010101E021F001012D
:1008C000816070470029816802D041F4807101E0A5
:1008D00021F48071816070472DE9F041824E92B021
:1008E000304600F00BF90BA800F039FA01214FF463
:1008F000C06003F0F9FA00248DF831404FF4602015
:10090000CDE90D044FF4A0204FF009080B9001270A
:100910008DF83C808DF830700BA9304600F080F9DE
:10092000724D8DF831408DF830708DF83C700BA908
:10093000284600F075F901231A460F21304600F0D1
:10094000C0F9022201231146304600F0BAF9012312
:1009500003220021304600F0B4F901230422194695
:10096000304600F0AEF9012305220B21304600F09D
:10097000A8F9012306220421304600F0A2F9012340
:1009800007220821304600F09CF9012308220321A8
:10099000304600F096F9012309220A21304600F082
:1009A00090F90121304600F084F90121284600F039
:1009B00080F901231A460521304600F055F901233C
:1009C0001A460621284600F04FF90021304600F073
:1009D000CBF84FF4E041284600F0C6F8012130463C
:1009E00000F0B8F80121284600F0B4F801213046A3
:1009F00000F0A6F80121284600F0A2F801213046B7
:100A000000F09EF90121284600F09AF940F61451B1
:100A1000374804F00EFE12208DF8400002208DF8B9
:100A200041008DF842408DF8437010A802F01AFF83
:100A300001224FF49061304600F0E8F80121304681
:100A4000FFF740FF01213046FFF732FF0121284622
:100A5000FFF72EFF304600F06EF9304600F09FF8A9
:100A60000028FAD1304600F075F9304600F082F8DF
:100A70000028FAD1284600F05EF9284600F08FF8E9
:100A80000028FAD1284600F065F9284600F072F8EF
:100A90000028FAD10121084603F002FA154D284634
:100AA00000F0A6FD684600F04EFE0F4801A94C304C
:100AB0000090114881E811018020CDE904404000F8
:100AC000069080000790202008904FF44050CDE918
:100AD00009046946284600F019FE0121284600F065
:100AE0007BFD12B0BDE8F0810024014000280140E8
:100AF000002C014008000240B00200200D4910B552
:100B0000884202D1012144150AE00B49884202D1F2
:100B10000121041504E0094988420AD10121CC03CE
:100B2000204603F0EDF92046BDE81040002103F017
:100B3000E7B910BD0024014000280140003C0140FD
:100B40000029816802D041F4801101E021F4801174
:100B5000816070470029816802D041F4004101E0C2
:100B600021F4004181607047826822F4E0420A4328
:100B700082607047014600208968490700D501203E
:100B8000704710B50246002054680B0AC9B20C40E9
:100B90001168194202D0002C00D0012010BD01467E
:100BA00000208968090700D50120704738B5012168
:100BB0001C2003F099F9FF20ADF8000000248DF807
:100BC000034003258DF8025069460D4801F0FAFAFA
:100BD0000120ADF800008DF803408DF80250694601
:100BE000084801F0EFFA2320ADF800008DF803402B
:100BF0008DF802506946044801F0E4FA38BD00005F
:100C000000080140000C014000100140002A426829
:100C1000C9B201D00A4300E08A4342607047000035
:100C200010B542680E4B0C791A400B6842EA042258
:100C30001343436083680B4A1340D1E902422243C5
:100C40004C7943EA44031A438260C26A097C22F465
:100C50007002491EC9B242EA0151C16210BD0000D2
:100C6000FFFEF0FFFDF7F1FF70B5072409290AD94F
:100C7000C568A1F10A0606EB4606B440A543B34099
:100C80001D43C56007E0056901EB4106B440A5437B
:100C9000B3401D430561836BC3F30154121B921CC7
:100CA00002EB82041F22A2409343A1400B438363C3
:100CB00070BD826B491E22F4401242EA01518163E9
:100CC000704770B5072409290AD9C568A1F10A0639
:100CD00006EB4606B440A543B3401D43C56007E09C
:100CE000056901EB4106B440A543B3401D430561CE
:100CF0001F23072A09D2446B521E02EB8202934043
:100D00009C4391400C43446370BD0D2A09D2046B8F
:100D1000D21F02EB820293409C4391400C43046338
:100D200070BDC46A0D3A02EB820293409C4391402D
:100D30000C43C46270BD816841F008018160704756
:100D40000029816802D041F4A00101E021F4A00152
:100D500081607047816841F0040181607047002123
:100D60000160017141718160C160012101747047AE
:100D700070B51E4C214694F83800B1F84250062850
:100D80001ED9B4F84A10B4F84C00A1EB000202F1ED
:100D90000902122A04D8FFF753FB0022144B0AE081
:100DA000884204D2FFF74CFB0022124B03E0FFF70E
:100DB00047FB0022104BFFF72CFAFFF786FB09E0F8
:100DC00005D12846FFF73CFB0C4A0D4BF3E70D49D4
:100DD00051F82000C5EB45116063B0EB410F03D91A
:100DE000C5EB45104000606370BD00004404002066
:100DF00000003440000033400000354067666666FE
:100E000066E64B40E88C000810B50C4C2078400793
:100E100013D5FFF7ADFF0A49A08E08800848303887
:100E2000018821F010010180001F018841F01001AC
:100E30000180207820F00400207010BD44040020C0
:100E400040040040F0B41448144B154A816804462D
:100E50001B782468526CCF0541F0080521F0080684
:100E60004FEA047413D5002C07DB090712D4002BBA
:100E700010D1142A0EDA856006E009070AD5002B86
:100E800008D1142A06DA8660F0BC05F093BD002C68
:100E9000F3DAEAE7F0BC7047A0020020F706002072
:100EA0004401002070B506464089204B204C4FF489
:100EB0008071002580B362887AB1012A0CD1E18863
:100EC000491C89B2E1803289914205D36580E58071
:100ED000FF2801D0401E708170BD7088228890422A
:100EE00001D9012200E00022184601F0F4F97088CF
:100EF000B18801442088401C80B220808142EBD818
:100F00002580A088401C80B2A080F1888842E3D36D
:100F100001206080A58070BDFFE70022184601F027
:100F2000DAF9A580E58025806580F4E7000C0140B2
:100F3000B4050020FEE70000FCB505464FF6FF763D
:100F400000200C46ADF8006048F205078DF804005B
:100F500020E000BF15F8010B8DF8040001A9084638
:100F600002F0E3F8BDF800009DF8041080EA0120CB
:100F7000ADF800005FF00000BDF800100A0402D5D3
:100F800087EA410101E006EA4101401CADF800108A
:100F90000828F1DB641EDDD26946084602F0AFF88E
:100FA000BDF80000FCBD00000246002004E000BFC8
:100FB00012F8013B1844C0B2491EF9D27047000034
:100FC00070B5144A85B01088002413490194009428
:100FD000039420460494138807E00D8B009E35444B
:100FE0000095CD8B019E3544019515889D42F4D026
:100FF000401CC0B28028EED30098411107484180C0
:10100000848001984111064881830183818205B063
:1010100070BD000000070020A0020020CE050020C7
:10102000BC04002030B50E4902880A800C4A43886F
:10103000083A13800B1F808818802024151F2C80ED
:101040000020401C80B27328FBD341F211100880AD
:1010500044F64800108047F2480018802C8030BDCC
:10106000202C0140114944F648000880091D46F62D
:1010700048000880091D41F2111008800B48001F2C
:10108000018841F02001018009480021A0F8641086
:10109000A0F86210A0F86010A0F85E10A0F85C1034
:1010A000A0F85A100348418181827047182C0140F2
:1010B000A002002068000020F0B54D4B4D480021F3
:1010C000DA7A0778802A27F001057CD31C684A4B1E
:1010D00002F01F0253F82220484B14421A6802D033
:1010E00042F0200201E022F02002454C1A60454EF9
:1010F00094F800C0444CBCF1020FB4F904403FD155
:10110000B3F808C0CCF3C00ECCF3002CE64537D0C2
:101110003A4D2C3D95F802C0BCF1000F04D0BCF153
:10112000010F0FD0A9702FE05FEA025C2CD55FEAB7
:10113000826C29D44FF0010C85F802C027F0040519
:10114000057021E05FEA025C1ED45FEA826C1BD569
:101150005FEA477C11D447F004070770B0F802C07B
:10116000BCF1000F03D0418027F0010704E0448068
:10117000002C02DD47F0010707700227AF7003E083
:1011800005704180318041811C4DC78895F84650DB
:101190000FB9002C15DC077BAF4212D1B0F90270F9
:1011A00007F26667BC420CDC184FBF895FEA477CD8
:1011B00007D45FEA877C04D45FEA427C01D5FF074D
:1011C0000BD0077800E00FE05FEAC77C05D027F07E
:1011D00001070770418031804181C4800573500947
:1011E00060F3CB221A60F0BD057041804181F0BDF3
:1011F000D40500200809002048910008A002002022
:10120000F706002018010020CE050020100A00205B
:101210002DE9F04796B000240C940D940E940F9491
:1012200072B69048816941F400718161816941F42D
:10123000806181614FF4004002F028FE8A4D002158
:101240002846FFF73FFB00212846FFF731FB874E7A
:1012500000213046FFF72CFB854F0021384600F077
:10126000BBF901204FF47041401C8842FCD3284652
:10127000FFF744FCB1463046FFF740FC384600F02B
:10128000B7F94FF46020CDE912048DF845400120F4
:101290004FF004088DF8440010948DF8508010A988
:1012A0002846FFF7BDFC01231A4605212846FFF713
:1012B00008FD0123022206212846FFF702FD012333
:1012C000032207212846FFF7FCFC012304220F21FB
:1012D0002846FFF7F6FC384600F08AF9684600F029
:1012E00032FA6148634E4C300090CDF80C80CDE965
:1012F00001648020CDE90440400006908000079002
:10130000202008904FF44050CDE909046946384642
:1013100000F0FCF901212846FFF7D4FA01213846F4
:1013200000F05AF901212846FFF7C2FA47F230517E
:1013300015941598401C15908842FAD3012128462F
:10134000FFF7FEFCADF82C40A04640F2DC5A4FF40B
:10135000007420E05046CDF854801599491C159131
:101360008142FAD330880D9908440D9070880E9907
:1013700008440E90B0880F9908440F90F0880C999B
:1013800008440C9001212846FFF7DAFCBDF82C0038
:10139000401CADF82C00BDF82C00A042DAD30D980B
:1013A000354A40F3CF1633480A3006830E9941F38D
:1013B000CF1444830F9941F3CF1383830C9941F3E6
:1013C000CF1CA0F804C0ACF5C05C40F2C371ACF512
:1013D0009B7C8C450ED2A6F5C856363E8E4209D26D
:1013E000A4F5C854363C8C4204D2A3F5C853363B0E
:1013F0008B4203D3D18841F48041D180D188490404
:1014000007D41E49028B21F85C2F428B4A80808BC7
:10141000888000212846FFF755FA0021384600F061
:10142000DBF800212846FFF743FA00214C464846E6
:10143000FFF73EFA0220C102401C8842FCD3284636
:10144000FFF75CFB2046FFF759FB384600F0D0F869
:10145000FFF742FA0A493C20087062B616B0BDE8B0
:10146000F0870000001002400024014000280140E5
:10147000080002401A050020100A0020640C002019
:10148000F4060020F0B5384B394C93F85650374BE2
:10149000042D5B6C1DD0256840F22D465D1B6560F8
:1014A00043F6FB25B3F5FA5F33DDB3F5FA4F30DCD5
:1014B00041F6AD17A3F5FA535F4306EBA7364FF499
:1014C000B5777B4305EBA31375105B10C4E9065396
:1014D00021E043F6D017102641F26205BB4218DB2B
:1014E00044F25067BB420EDAA3F5645345F24C67F1
:1014F000D03B5F4306EBA736A66140F624767343E4
:1015000005EB232303E042F24713A361194BE36188
:1015100001E0C4E90665A3695360E569401AD56036
:1015200010604543107C0541106A29181162D0698A
:10153000814200DD1062116A9069814201DB084638
:1015400000E01062206211684B43117A0B410841A0
:101550001918B2F91400884204DBB2F9120088426B
:1015600000DC08B2F0BD000068000020440100204B
:101570001C01002085EB010010B54FF400542046FB
:1015800000F0ACF8002813D00A49087840F00800B1
:101590000870204600F014F80021074800F01CF8FD
:1015A0000648C17E012903D10021C17601210177BE
:1015B00010BD00006E06002044000240080B002011
:1015C000C10002D50249086070470249486070476F
:1015D00004040240000002400029016802D041F0EA
:1015E000010102E04FF6FE721140016070470000F9
:1015F00001684FF6FE7211400160002101604160F8
:101600008160C1603149314A0839904203D148684C
:1016100040F00F0006E02D4A1432904204D1486891
:1016200040F0F00048607047284A2832904203D1C9
:10163000486840F47060F5E7244A3C32904203D198
:10164000486840F47040EDE7204A5032904203D1A0
:10165000486840F47020E5E71C4A6432904203D1A8
:10166000486840F47000DDE7184A7832904203D1B0
:10167000486840F07060D5E7154A111F904203D1C9
:10168000086840F00F0006E0114A1432904204D17D
:10169000086840F0F000086070470D4A2832904218
:1016A00003D1086840F47060F5E7094A3C32904283
:1016B00003D1086840F47040EDE7054A503290428B
:1016C000EAD1086840F47020E5E700000800024015
:1016D00008040240406880B27047000001460020C4
:1016E000CA0001D5034A00E0034A12680A4200D04A
:1016F000012070470004024000000240002A0268F6
:1017000001D00A4300E08A430260704730B50368A5
:1017100047F6F07293430C6A8A682243D1E9044584
:101720002C4322438C692243CC6922434C6A2243D6
:101730008C6A22431A430260CA6842600A68826067
:101740004968C16030BD0021016041608160C160B5
:10175000016141618161C1610162416281627047E1
:1017600010B5114C8CB000212046FFF735FF204604
:10177000FFF73EFF0D4800900D480021CDE9010123
:101780006420CDE903018020CDE90501079108918E
:1017900009910A9169462046FFF7B8FF01212046CA
:1017A000FFF71AFF0CB010BD58000240043801408A
:1017B0008C07002010B501218CB0084602F070FBA8
:1017C0001E4C00212046FFF707FF2046FFF710FFC1
:1017D0001B4800901B48019000211020CDE9020118
:1017E0008020CDE9041006910791089109910A9192
:1017F00069462046FFF78AFF012202212046FFF7B3
:101800007DFF01218DF82F1004208DF82D008DF81B
:101810002E100E208DF82C000BA802F023F80F20BC
:101820008DF82C000BA802F01DF801212046FFF7CF
:10183000D3FEFFF795FF0CB010BD0000440002403E
:10184000043801402807002030B540F6AA21204A7C
:10185000C184838B1488E31A9BB20F2B10D3128898
:101860008283037E002253B11A4BB3F90A30062B50
:1018700005DB194B1B78022B03D0002B00D182848F
:1018800030BD164B40F68B255B6CA3F22D14AC4299
:101890000FD2428B521C92B24283642AF0D364224C
:1018A0004283B0F924208A4201DA02EB21118184BB
:1018B00030BD41F29414A342FADBB0F92430002B7E
:1018C00002DDA3EB211100E000218184428330BDC1
:1018D0000007002068000020F706002044010020D7
:1018E00010B50446B0F9020043F69911484381133C
:1018F000E06840F26662504301EBA030E060B4F96A
:10190000001043F6991251438A13216940F266632D
:10191000594302EBA131216104F0B2FC6061A1885E
:1019200040F6AB2208444010A0F515415539E0625D
:10193000914205D9A0F5F851FF39521C91421DD2B0
:1019400049F25451884202DDA0F5204002E0A0F5A2
:10195000F850FF38206300EB400040F34F00208533
:10196000B4F924104A42904201DA104602E088425B
:1019700000DD0846E083228461848AE0A0F5FE420F
:10198000FF3A41F255518A4214D8A2F6AA202063A8
:1019900000EB400040F34F002085B4F92420514271
:1019A000E183884201DA084602E0904200DD1046F9
:1019B000404250E0A0F5D442AA3A8A4215D2A2F69B
:1019C000AA20206300EB400040F34F012185B4F9C9
:1019D00024004242E2832084914201DA104602E070
:1019E000814200DC0846608453E0A0F5AA42543AE4
:1019F00041F256539A4215D2A2F6AB20206300EB77
:101A0000400040F34F002085B4F924104A42904230
:101A100001DA104602E0884200DD08464042E083D9
:101A2000218419E0A0F5804241F254539A4215D224
:101A3000A2F6AA20206300EB400040F34F0121856D
:101A4000B4F92400E0834242914201DA104602E0F8
:101A5000814200DC0846208462841AE0A0F5285206
:101A6000AB3A8A4215D2A2F6AA20206300EB4000CE
:101A700040F34F012185B4F92400E08342422284DF
:101A8000914201DA104602E0814200DC0846404201
:101A9000A9E7B4F91E006FF4BF7148438013E080DA
:101AA000B4F92000484380132081B4F92200484350
:101AB0008013608110BD70471548164A4FF480416D
:101AC0000078042821D002F13C03D08A9B88C01AF8
:101AD00000B22F2801DD001108E0002801DD002000
:101AE00007E00D4B984201DA184602E0402800DD7D
:101AF00040209389184400B2884203DC40F26661BA
:101B0000884200DA08469081704791817047000052
:101B1000F7060020BC040020C0FEFFFF38B54B488C
:101B20004B4902880B889A1A92B20F2A71D30988FE
:101B3000484C01804FF0FF01E2884FF47A7355045E
:101B40004FF4967002D51622009103E0950403D558
:101B500015220091014670E0D50402D514220091AF
:101B6000F8E7150502D513220091F3E7550502D5D4
:101B700012220091EEE7950502D511220091E9E7C6
:101B8000D50502D510220091E4E7150602D50F22F3
:101B90000091DFE7550602D50E220091DAE795069F
:101BA00002D50D220091D5E7D50602D50C22009171
:101BB000D0E7150702D50B220091CBE7550702D5D8
:101BC0000A220091C6E7950702D509220091C1E7D4
:101BD000D20702D008220091BCE72289550702D51E
:101BE00007220091B6E7950702D506220091B1E7DA
:101BF000D20702D005220091ACE7A27AD20702D028
:101C000004220091A6E7A289D40603D503220091FD
:101C1000A0E719E0140702D5022200919AE75407C1
:101C200003D4940701D4D20702D00122009191E796
:101C30000020034602460146009002F00BFEBDE87C
:101C400038400248FFF72EB938BD0000040A0020D2
:101C500000070020100A0020F0B559485949828831
:101C60000B889A1A92B29C2A64D3098881805649BB
:101C70000A880146002A0B7843F0020156D1164625
:101C8000524A1C0715680246127822F0020274D5E7
:101C90004F4C0746E4887F785FEA845C02D547F0C2
:101CA000010701E027F001074770A704477802D534
:101CB00047F0020701E027F002074770670401D4EC
:101CC000E70703D0477847F008074770640603D555
:101CD000447844F0040404E01C0603D4447824F05F
:101CE00004044470EC0450D4354C9A07247824F052
:101CF000100423D4324D42782F7A2D78012A45F0F2
:101D0000100514D0022A16D02D4C042AA47804F110
:101D1000010C0CF0FF0C13D0072A25D0032A23D086
:101D2000052A21D0062A1FD021F0100142E0B90770
:101D300002E00570F0BD39070029FADB0470F0BD40
:101D4000FA0601D41A060AD50170022C04D280F8D2
:101D500002C0BCF1020FF2D341F080012AE021F071
:101D6000100101708670F0BD877A7F06F7D5032CCD
:101D700004D8017080F802C0F0BD0FE05107D8D53B
:101D80001906D6D443F0800114E002704178CB07E5
:101D900001D18907F0D522F010010BE0E9040BD442
:101DA0009907E9D4818AC82902D2491C8182E3E7D4
:101DB00043F00A010170DFE702708682DCE7000071
:101DC000D80600200007002002070020A002002003
:101DD000100A0020094944F648000880091D46F60B
:101DE00048000880091D41F6CC4008800348001FC8
:101DF000018841F02001018070470000182C01404B
:101E0000084946F668000880091D0880091D41F24E
:101E1000555008800348001F018841F020010180CF
:101E200070470000182C014010B5C28800210AB18B
:101E3000032206E002890AB1022202E0428912B1BD
:101E40000122027000E0017004784FF4804344F6F0
:101E5000206244B1012C06D0022C07D0032C01D102
:101E60004180818010BD4380828010BD41F23331BA
:101E7000418040F6B731F4E730B5B1F86A5000233D
:101E80001A240D22854202DCB1F9680030BD4D886C
:101E9000854202DBB1F9000030BD01EB82056D889F
:101EA000854201DD144601E013DA134604EB030218
:101EB0004FEA52029A42F0D101EB830231F823102B
:101EC00054889288521A001B424301EB622000B2F0
:101ED00030BD31F9220030BD054920B1086940F01C
:101EE00080000861704703484860034848607047B5
:101EF0000020024023016745AB89EFCD06494FF42E
:101F00007A70CA68D20705D0401E0004000CF8D1D0
:101F1000FF20704700207047002002401248032134
:101F2000A0F1540280F83610002111820F4A118668
:101F30000F4A1186D162D1831184518481620D4987
:101F40008A6CB2F5206F01DBA3228262897A11B11B
:101F5000816A49428162C16A41F3910181628803C9
:101F6000054908627047000068000020A0020020B8
:101F700024050020440100206C080020F0B53B49F6
:101F800088894A89801A80B20F2866D38889488157
:101F9000CA8937480B3A272A26D28A7822BB826818
:101FA000364B42F480728260324A354C354D12789D
:101FB0005607314A0AD4344E36881680334A12887E
:101FC0001A80334A12882280324A09E0324E36881B
:101FD0001680324A12881A80314A12882280314A89
:101FE00012882A8001228A702F4B304D19469A7F21
:101FF0000968802A32D302F01F0255F822201142CC
:102000002CD0826822F48012184E82601236144658
:102010001215B778521C62F38617254AB77093F8E9
:1020200016C01778BCF1800F27F0020608D30CF019
:102030001F0C55F82CC011EA0C0F01D147F0020615
:1020400016701A7E802A0DD302F01F0255F8222046
:10205000114207D144F400218160F0BD826842F44E
:102060008012D1E724F40021F6E70000F4060020F6
:10207000A002002044010020B4040020B604002087
:10208000B8040020BA040020A4040020A604002004
:10209000A8040020AA040020AC040020AE04002004
:1020A000B0040020B2040020D405002048910008AC
:1020B000BC04002070B5204881890289891A89B240
:1020C0000F292FD3818901811C4B1D4819465D7A48
:1020D00006681C4C096846F00402802D07D305F001
:1020E0001F0554F82550294201D126F00402026050
:1020F0009A7B802A17D302F01F0254F82220114243
:1021000011D1026822F002020260DA7A802A0ED32C
:1021100002F01F0254F82220114208D1016821F078
:102120000801016070BD026842F00202ECE701683C
:1021300041F00801F5E70000F4060020D405002076
:10214000A002002048910008F0B51D4C1B4A4FF03A
:10215000010C94F83B5094F80AE0144692F83C3095
:1021600094F838402B43651CEEB2154D95F83D7040
:102170000025BEF1FF0F0AD0BEF1000F06D18B4241
:1021800013D155700C2C01D282F83860F0BD834217
:1021900002D182F801C0F5E78B42F7D15570B8073C
:1021A00009E000BF82F83850F0BD8342FCD1F8430B
:1021B00082F801C080070028F4D0F0BD440400205C
:1021C00044010020F0B5CA78002502F00F03D206C2
:1021D00001D58A7813430A784FF00F0E12F0FF0FE3
:1021E0004FF001021CD004680F8802FA05F6374050
:1021F000B74211D14FEA850C0EFA0CF724EA070713
:1022000003FA0CF43C43CF78282F02D0482F02D099
:1022100002E0466100E006616D1C082DE4D3046015
:102220000C88FF2C1ED944685FF0000606F10807F1
:1022300002FA07F50F882F40AF420FD14FEA860C04
:102240000EFA0CF7BC4303FA0CF73C43CF78282F67
:1022500000D14561CF78482F00D10561761C082E4A
:10226000E4D34460F0BD0000F0B5144C002801DA5E
:10227000E36900E06368420D120185B2C0F30157C3
:102280009540C0F30346032F05D0C2020AD50322AE
:10229000B240934307E023F07062636823F07063F9
:1022A000636002E0AB4343F0706201B12A4300284F
:1022B00001DAE261F0BD6260F0BD000000000140A3
:1022C0000246002092680A4200D001207047416116
:1022D0007047016170470AB1016170474161704701
:1022E0000F4A104B92F838105B5C834201D10120F9
:1022F00004E00D4B5B5C834203D1002082F83A007E
:1023000070470A4B5B5C834201D18120F6E7084BA2
:10231000595C814201D18020F0E70320EEE7000004
:1023200044010020089500081A9500080E95000841
:10233000209500080A4810B501784FF000024C07BC
:1023400008494FF0FF0389684FEA017105D500295C
:1023500001DA827210BD837210BD0029FBDBF8E741
:1023600044010020A0020020F0B5194E194C0022B3
:10237000E31CA6F1060CB75CA518ED78FF5C0D43D5
:102380000F43BD421FD01CF80270FF5C0F43BD42DB
:1023900019D015460023A618F6780E43C6545B1CC8
:1023A0001CF80220DBB2062BF5D3C17881700179CD
:1023B000C17000214218491C15711CF80550C9B2A2
:1023C0000629F7D3F0BD521CD2B2032AD3D3F0BDF5
:1023D000DA8C00084404002010B502460021064BA8
:1023E00006205C186478944200D10846491CC9B2A2
:1023F0000629F6D310BD000044010020214810B585
:1024000090F8671000222048012936D11F49898899
:1024100099BB1F491E4B4C6C40F6B831B3F86E3077
:102420008C4227DD1B49097821BB90F82711491CF4
:10243000C9B280F82711C8291CD380F8272101468A
:10244000D0F82C4191F82811A34203DD052908D2C8
:10245000491C01E041B1491E80F82811C9B2052983
:1024600002D3012180F82611191B074C2C3C616214
:10247000C0F82C31B3F5FA6F03D280F8262180F82A
:10248000282110BD640C0020A0020020CE050020F1
:1024900044010020F70600204FF4C0428260002172
:1024A00041620E22828141F262020261082282822E
:1024B0004FF46042C28201834FF07842C0E90721A5
:1024C00040F6C41101807047B0F90010B0F9022045
:1024D000891A41600269037D4A431A41436A1344E1
:1024E0004362026A934200DD4262436AC2699342D8
:1024F00000DA42628268436A4A43017B0A410B4127
:10250000D118B0F918208A4201DA10467047B0F9A4
:1025100016008842FADC08B27047000010B5144873
:102520001449B0F88C200B889A1A92B2B2F5437F06
:102530001DD90988A0F88C10B0F88A1020F8581F0F
:10254000002242860C480D4CC2888280C180C3891B
:1025500083812489891AA4B2C4818160E11A01614E
:10256000074A818AC182928A8282511A816110BD92
:1025700044010020000700202C0C0020240500202E
:102580006800002009480A49B0F8AA200B889A1A66
:1025900092B241F684639A4206D3098820F8AA1FB2
:1025A0004188818000214180704700004401002063
:1025B000000700200D480178C90702D00C4909889E
:1025C00001E04FF6FA71C165094901201039088010
:1025D00007482438018841F0010101800448183877
:1025E000018821F01801018070470000440100209B
:1025F000240400400A49D1F8902012B1521EC1F8BB
:10260000902031F88A2F521C21F81A294A6A521C4C
:102610004A628A8F521C8A8701F8380C7047000082
:10262000440100201CB52D4890F83B3090F83C2028
:10263000934252D000248DF8044053408DF800306E
:102640009DF800300122012B08D09DF80030022BAC
:1026500009D09DF80030042B0AD00DE01F498DF8F9
:102660000420443108E01D498DF80420463103E080
:102670001A498DF8042048319DF80420012A2CD1F4
:1026800090F83D309DF80040154AA34217D090F8CD
:102690003E309DF80040234208D0B0F84C30A0F8FE
:1026A0004A300B881488E31AA0F84C3090F8383080
:1026B0002BB1B0F840301488E31AA0F842301288E9
:1026C0000A80A0F8402010F83E1F9DF8002011431A
:1026D00000F801199DF8001001701CBD4404002091
:1026E0000007002070B5344D40212846FFF7E8FD73
:1026F000840080212846FFF7E3FD44EA4004A91541
:102700002846FFF7DDFD0443E1B22C4C94F87050ED
:102710008D4250D04D4084F87010012D03D0022D11
:1027200001D0042D47D194F87400A84384F87400B4
:1027300094F87320AA420FD084F8735094F8722052
:1027400001238B401A4207D11A4384F8722094F86F
:102750007110491C84F8711094F87110042928D361
:1027600030B1012811D002280FD004280DD012E07A
:102770001348C18821F04001C1802078002184F8ED
:102780003B1020F06000207005E0217841F020012E
:10279000217084F83B000B4994F83B0091F8272006
:1027A000904204D081F8270007492020087000F0EB
:1027B0000DF884F84C5070BD001001404401002019
:1027C000100A0020640C0020F406002070B50D4DA6
:1027D00040212846FFF774FD840080212846FFF73A
:1027E0006FFD44EA4004A9152846FFF769FD04433C
:1027F0000548072100F8704F017100214170817078
:10280000C17070BD001001404401002070B5344813
:1028100090F83A10CA43920761D001F0030280F8A1
:10282000392090F83D305B061B0E80F83D30012AC0
:1028300001D0812A02D15B1C80F83D300278D2079A
:102840004DD0DBB203F00102C3F34004A24246D1F3
:10285000B0F84E400025641CA0F84E40204CA0F873
:10286000505090F83E60A47AB24202D080F83E20E8
:102870000DE0A607B6EB837F02D080F83F5006E05C
:1028800090F83F30642B02D25B1C80F83F3090F808
:102890004030642B0CD25B1CDBB280F84030022B42
:1028A00006D204F00103934202D1022280F84020B4
:1028B000012901D0002912D190F83820C16D00EB18
:1028C000820291610163D0E906121144D0E9082324
:1028D0001A441144826A1144C26A1144416370BDB2
:1028E00044010020FEE700002DE9F04F00BF00206A
:1028F0009E4E9F4AA6F51271A6F5BE79A6F1440B2D
:1029000006F1440E804601F5E074A1F1780301F56B
:10291000457A1D5C15F0C00706D0402F51D0C02F5E
:1029200077D0802F76D004E115F01F0504D0154430
:1029300040F080072F7201E082F80880012826D03D
:10294000022824D0032822D0042820D008281ED012
:1029500010281CD0874D55F820C0DCF8005054F8E2
:1029600020703D40CCF80050824D55F820C0DCF876
:10297000005056F820703D43CCF800501D5CAD0669
:1029800059F820502F6813D53AF810C03EE051F89E
:1029900020502F6854F820C007EA0C072F6051F828
:1029A00020502F6856F820C047EA0C072F60E5E753
:1029B000DFF8B8C10CF1F00C5CF820C007EA0C0796
:1029C0007EE015F01F0504D0154440F080072F72FB
:1029D00001E082F8088001281DD002281BD00328BE
:1029E00019D0042817D0082815D0102813D0614D0D
:1029F00055F820502F6854F820C007EA0C072F60C4
:102A00005C4D55F820502F685BF820C047EA0C0752
:102A100056E00BE056E051F820502F6854F820C0E3
:102A200007EA0C072F6051F82050ECE715F01F055E
:102A300005D0154440F0800785F8217001E082F848
:102A40002180012825D0022823D0032821D0042862
:102A50001FD008281DD010281BD0464D55F820C087
:102A6000DCF8005054F820703D40CCF80050414D47
:102A700055F820C0DCF800505EF820703D43CCF8DB
:102A800000501D5CAD0615D53A4D3AF81070CC35A6
:102A900014E051F820502F6854F820C007EA0C07C2
:102AA0002F6051F820502F685EF820C047EA0C07CD
:102AB0002F60E6E72D4D3AF81070E03D55F82050B4
:102AC0002F6036E015F01F0505D0154440F0800753
:102AD00085F8217001E082F82180012830D0022899
:102AE0002ED003282CD004282AD0082828D010283B
:102AF00026D0204D55F820C0DCF8005054F8207046
:102B00003D40CCF800501B4D55F820C0DCF800507B
:102B1000164F883757F820703D43CCF800501D5CA5
:102B2000AD06B1D4114F3AF81050E03F57F820707D
:102B30003D60401CC0B21128FFF4EBAEBDE8F08F41
:102B400051F820502F6854F820C007EA0C072F6076
:102B500051F820502F68DFF814C00CF1880C5CF895
:102B600020C047EA0C072F60D9E70000D493000883
:102B7000D4050020D09100084FF40771C1824FF4B2
:102B80005861018340F6145181837047F0B5C48ABF
:102B9000B0F900608681B0F90250C581B0F9043007
:102BA0000227002101220382AB4204DBB54202DD91
:102BB000C78042810CE0B34204DBAE4202DDC78035
:102BC00041811CE09D4205DBB34203DDC2804781A9
:102BD000018115E0B54204DB9E4202DDC2804181E5
:102BE00005E0AE4205DB9D4203DDC18042810781E5
:102BF00006E09E4204DBAB4202DDC18047810281D8
:102C0000C388458900EB430700EB4505BB89AE89C6
:102C10009B1B0FFA83FEA0F812E00689AB8900EB3C
:102C2000460CBCF80CC0A3EB0C038382B0F918303F
:102C3000B7F90CC0A3EB0C0CB4EB4C0F04DA80F822
:102C40002010A3F1A10113E0A64503DD80F82010B8
:102C5000B9890BE026B1012E04D0022E10D004E079
:102C6000062100E0052180F82010A989091B6D319B
:102C7000418309B2B1F5586F04DB5B1E438304E066
:102C80000421F0E7002900DC4283418B8183F0BD01
:102C90000B49002288760A62CA614A62094A32F9FF
:102CA000103002EB40028B62B2F90220CA62064A7F
:102CB00032F810000882A1F86000A1F862007047A5
:102CC000F401002032950008269500082DE9F05FF8
:102CD000F848F94982880B889A1A92B20F2A44D38D
:102CE00009888180F549824601270888F44CF54E11
:102CF000002578B3401E0880E573F349A56220687B
:102D0000B1F90210430742F6AA2218D4F38843F41B
:102D10000053F380EC4B1B789B0709D5A36823F085
:102D20008003A360A4F87C5084F87E5084F87F5020
:102D3000C30404D484F8F070C4F8EC5003E084F8C1
:102D4000F050430707D4914205DB84F8F470A4F8EF
:102D5000F25004E010E084F8F450430703D49142A9
:102D600001DBC00703D084F81151BDE8F09F84F85F
:102D70001171A4F81251F8E7B4F8180143F698213C
:102D8000884202D2401CA4F8180101F079FDDFF856
:102D90003C83DFF820B398F85000ABF1180B10B16A
:102DA000FEF78AF905E09BF8001021F001018BF88D
:102DB000001098F8630010B1FEF744F808E0A0682E
:102DC000C10502D520F0080001E040F00800A06035
:102DD000FFF714FB00F0C0F9BD4841F26801436CF5
:102DE0004FF400608B4201DBBA4904E0B3F57A6F1F
:102DF00002DAB849091D086098F85100C646C107B3
:102E0000DFF8BC82B448DFF8D492A8F12C0839D09E
:102E1000817B802932D3217889072FD4E17B88F800
:102E20000510A949424691F800C02CF0020C81F827
:102E300000C0ABF80250CBF814509BF800C02CF047
:102E4000010C8BF800C0B179490612D4518941F2C6
:102E5000883C614503D2491CA8F80A1012E040F6EC
:102E60003C70834201DD0020F9E0042088F8037003
:102E7000F5E0D5700020A8F80A50F0E088F803507B
:102E8000A8F80A50A1680A0501D50820E7E09EF8D5
:102E90003FE05FEACE7240D0E27B88F80520437ABB
:102EA000802B5BD323785B0730D4F3889B0403D556
:102EB00021F02000A06030E0ABF80250CBF81450B5
:102EC0009BF800C041F020012CF0010C8BF800C0F1
:102ED000A160C17D802909D301F07F0300684FF014
:102EE0000041D940084201D1277100E025712079C5
:102EF000C00702D15FEA8E7005D50320032A01D0F6
:102F000088F80870ABE00020A562A8E021F020005E
:102F1000A060F08820F40050F08094F82601012889
:102F200021D094F846104FF48047F1B143F2333288
:102F3000012932D0032999F80010694843F6991302
:102F4000C1F381012CD0012941D002293FD090F852
:102F50005600042838D0A4F814713EE0206840F0F0
:102F600004002060A4E7092079E099F8000042F607
:102F7000CC41C0F38100012809D002280AD042F6D2
:102F8000B86000BFA4F81401A4F8441027E0A4F826
:102F90001411F9E742F26660F4E7A4F814211CE08A
:102FA00001290AD0022908D090F8560004280BD035
:102FB000A4F81431A4F8447011E0A4F8147190F846
:102FC0005600042814D0F5E7A4F8147110E0A4F812
:102FD000147190F8560004280AD0A4F84420FEF793
:102FE0006BF89BF80010C90705D0BBF8021004E08D
:102FF000A4F84430F3E734488188AAF8121008B2E4
:10300000B4F944104843C0F38F314046A8F8121079
:10301000B94200D9478233490978C90605D5428AA1
:1030200041F233318A4200D241822189C1F3C00288
:10303000C1F300218A4205D1428A40F6CC418A423E
:1030400000D94182B17AC90700D04582B8F8120090
:10305000A06200287FF707AF2348057002209AF886
:103060001A1099B9022841D080B119490B789D06F0
:1030700008D5B5796D0605D51A4D2D78ED0965F39E
:1030800086130B70F18821F40A61F1801049496CB4
:103090004E290ADBF1880B0607D521F08001F1806B
:1030A00009490B7823F002030B708AF81A00E073C9
:1030B0005BE6000020090020000700200207002036
:1030C000A0020020100A0020CE050020640C002081
:1030D00044010020100C0140D4050020BC04002055
:1030E00068000020D806002014070020B9F8383006
:1030F000002BBAD143F69823A9F83830B5E770B55C
:1031000000230C8863F30F02012505FA03F634420D
:1031100006D0C3F10F0605FA06F1114361F30F0261
:103120005B1C102BF1DB028070BD70B500230C78A6
:1031300063F30702012505FA03F6344206D0C3F112
:10314000070605FA06F1114361F307025B1C082B21
:10315000F1DB027070BD0000F0B51F4890F86630DA
:103160001E48012B816821F4006232D11C4BDE889D
:1031700074062ED41B4D0F054FF00004B5F9025014
:103180001ED4194A526C642A11DC40F6386295420A
:103190000DDAB2040BD4027852070ED4B0F8D42062
:1031A00040F6B835AA4203D2521CA0F8D420F0BD94
:1031B00041F4006181605C81F0BDA0F8D440F0BDB5
:1031C00041F2CD018D42FADD997AC907F7D18260CB
:1031D000F3E78260F0BD0000640C0020A002002034
:1031E000100A0020CE05002044010020F0B5364D25
:1031F000364F044695F83B0097F83B102378084378
:10320000EE1C6278834205D1E0781146FEF79CFF00
:10321000207908E094F802C084450CD1E17810468A
:10322000FEF792FFE07905F82F0F2878805D68702F
:10323000287BE877F0BD82421DD161461846FEF733
:1032400083FF95F84E1095F83B00814207D1B97A7B
:1032500009B1A17900E0617985F82F101EE0697845
:10326000012901D0A17922E0617927E0297841F094
:103270000401297012E0E1788142DBD119466046F1
:10328000FEF762FF95F84E1095F83B0081420AD197
:10329000B97A09B1617ADFE7217ADDE715F82F1FE6
:1032A000895D6970C5E76978012906D0617A85F87A
:1032B0002F10B97A0029F1D1D8E7217A85F82F109B
:1032C000B97A0029EAD0D1E7440400204401002063
:1032D0000B48017821F0020100F8381B002100F8AA
:1032E00018194177817733218185418508214184EF
:1032F000012100F81F1C034880F8391070470000B6
:1033000044040020440100200D4900B50B4851F849
:10331000012F40F8032F8988818008480121093056
:10332000FFF722F8054802211330FFF71DF8034884
:1033300004211D305DF804EBFFF716B844040020AB
:1033400044010020094944F648000880091D46F65A
:1033500048000880091D41F2111008800348001F31
:10336000018841F02001018070470000182C0140C5
:103370002DE9F047664C674B0025A0780126654A89
:10338000103305287ED2DFE800F00313113E110050
:10339000108820F0010010801D805F480580001F0C
:1033A0000580001F0580FFF7CDFFA670BDE8F08700
:1033B000594941F244401C390880574945F65800A4
:1033C00024390880091D47F25800088052492020FE
:1033D000283908800020401CC0B27328FBD3FFF7B7
:1033E000B1FF4C4984F85C502C3147F6906008805E
:1033F0004848143006801D80108840F0010010807D
:103400000220A070D2E700215FF0010004EB41022E
:1034100004EB4003B2F85020B3F850309A4200D287
:103420000146401CC0B20628F0D33C48405C84F8FA
:103430003900FFF74DFF1D2000F0F3F900F076F89A
:10344000374E38484FF4807996F83B10012904D064
:1034500002291BD0042930D047E040218046FEF7E6
:103460002FFF870080214046FEF72AFF47EA4007EA
:1034700049464046FEF724FF074347F0010084F821
:103480003B0000E03DE0224809302CE0402180462E
:10349000FEF716FF870080214046FEF711FF47EA3E
:1034A000400749464046FEF70BFF074347F002003E
:1034B00084F83B001648133015E040218046FEF7A3
:1034C000FFFE870080214046FEF7FAFE47EA4007EC
:1034D00049464046FEF7F4FE074347F0040084F8EF
:1034E0003B000B481D3002F0A5FD94F82F0086F834
:1034F00038001D2000F0ABF90420A0700A480570C8
:1035000054E7108820F0010010801D80A5704DE761
:1035100044040020000800403C2C0140E08C0008DE
:103520004401002000100140F70600202DE9F04181
:10353000344C14F82F0F344DE07240212846FEF72A
:10354000BFFE860080212846FEF7BAFE46EA400606
:10355000AF1539462846FEF7B3FE0643207BF1B28D
:103560002F3C814215D084F83C0040212846FEF7CC
:10357000A7FE860080212846FEF7A2FE46EA400606
:1035800039462846FEF79CFE064384F83B60FFF769
:1035900049F81E4D95F83B00012827D0022828D075
:1035A000042829D0174894F83B102730085C04F809
:1035B000300F14F80109FEF70FFF04F82F09A87A5D
:1035C00000B10120607001F0E7F994F84E0094F822
:1035D0003B10884206D094F83800062802D2401CDE
:1035E00084F8380084F84E10BDE8F08105480930B1
:1035F00004E00448133001E002481D30BDE8F0410A
:10360000FFF7F4BD440400200010014044010020F5
:103610002DE9F041524991F87200AA287ED191F823
:10362000730055287AD14F4C00200A5C2254401C6C
:10363000C0B27428F9D34C4E2069C6F80100A08AA4
:10364000A6F80500D4F81600F060D4F81A0030612E
:10365000D4F81E001234706102F092FC4349608A73
:10366000888102F0A7FC207D123CC007307802D090
:1036700040F0040001E020F004003D4930704FF4B8
:1036800080403C4D886114F8280F85F82000608B3D
:103690006880A08BA880E08BE880208C2881608CDB
:1036A000354F688194F8240087F8D20014F8011C83
:1036B000304686F83B100026C0F89460FFF724FEE1
:1036C0002E48A18E0183E18E4183218F818394F85E
:1036D0004210283C012908D0022901D0032909D031
:1036E000297821F00C01083107E0297821F00C013C
:1036F000091D02E0297841F00C01297094F86E2030
:10370000012162B1012A01D0022A0BD087F84610AC
:1037100094F864301A4A4BB1518108E014E087F8FC
:103720004660F5E7022287F84620F1E7568194F8D3
:10373000701001290AD094F86D1051B101290BD0F5
:103740004FF48051A0F87610BDE8F08144F21C716E
:10375000F8E74FF40051F5E741F25551F2E7000068
:1037600000FC0008640C00204401002068000020D8
:10377000FC0B0020BC040020A00200202405002037
:10378000100A00207CB50121082000F0ADFB4FF4A9
:103790008070ADF8040010248DF8074001208DF8EA
:1037A000060001A91548FEF70DFD0121092000F0D2
:1037B0009BFB01211248FEF757FD0820ADF80000E1
:1037C00004208DF803000F4E03258DF80250694642
:1037D0003046FEF7F7FC08213046FEF778FDADF8DD
:1037E00000408DF803408DF8025069463046FEF7E0
:1037F000E9FC10213046FEF76AFD7CBD0014014053
:1038000000023000000C0140FEE7704700F01F028C
:10381000012191404009800000F1E020C0F88011B2
:10382000704700F01F02012191404009800000F123
:10383000E020C0F88011704700F01F020121914084
:103840004009800000F1E020C0F80011704700F04E
:103850001F02012191404009800000F1E020C0F8E2
:103860000011704770B50F23C47801780122F4B1BC
:10387000144C2468457804F4E064C4F5E064240A38
:10388000C4F10406E3408478B5401C402C4301F1A8
:10389000E021230181F80034007800F01F018A4004
:1038A0004009800000F1E020C0F8002170BD01F067
:1038B0001F0082404809800000F1E020C0F880210C
:1038C00070BD00000CED00E00249084302490860A9
:1038D000704700000000FA050CED00E02DE9F05FF4
:1038E00000261D20FFF792FF6C4CDFF8B4B1A4F165
:1038F000B000A77E90F83810DFF8A8E1DFF8A8A1A3
:1039000000258F427ED0E776A176626A036B5A4328
:103910004FEA12499BF80820120702D51EF8012031
:1039200000E00A4694F812C0BCF1010F09D004EB84
:103930004206B6F902C0C4F828C0B6F90460E662CF
:103940000CE043F6FF7CC4E90A5C90F83DC05FEAF6
:10395000CC7C01D012B102E0052A00D1012600EB97
:1039600047074FF0804CBF893F04B7FBF3F3E36197
:10397000476BBCFBF7F7276294F813C0BCF1000F4C
:1039800006D0BCF1010F05D03B4403EBD3735B10B1
:10399000636201E03B466762DFF810C14FF6FF77D4
:1039A00007EA8307ACF808709AF8007090F80A806C
:1039B00090F83DC0082F08F003070CF0030C05D069
:1039C00067450BD1B8F1000F05D008E0674505D079
:1039D000B8F1000F03D05B42636200E06562C6B1DC
:1039E000636A002B03D006DD228D05E00AE0304B30
:1039F00033F8122000E0A28DA4F86020227822F093
:103A0000200222709AF80020042A07D0082A05D044
:103A100012E0B4F8603003EB0902EDE780F84050A3
:103A200065629BF80800000701D51EF801102048C8
:103A300030F81100A4F860001E49606A09883E3120
:103A40004843B4F8601001EB204006B21D20FFF798
:103A5000F3FE606A002807D021784FEA81600ADD12
:103A6000002804DAA08D09E0B4F8600006E0E06AFE
:103A7000B04208DB0CE0002802DA208D208208E04A
:103A8000A06AB04204DD208241F02000207000E0F6
:103A90002682257565752586BDE8F09FF401002016
:103AA000A002002014950008F7060020E809002075
:103AB000269500082404004043184FF480429342A6
:103AC00010DD904202DD104600210BE0914202DD44
:103AD0000020114606E08003B0FBF3F000B2C0F511
:103AE000804109B241EA0040704700002DE9F043EF
:103AF000002340F2AE440E2544600362058144F287
:103B00004C260827C6600782DFF8349043F6FF7C16
:103B1000A0F81290A0F814C04FF070484FEA8C3211
:103B2000C0E906824C600B620D81CE600F82A1F865
:103B30001290A1F814C0C1E90682BDE8F08300002C
:103B400000C0FFFF00214162094981600E2181818F
:103B50004FF6BF510161082181824FF44041C1827B
:103B600043F6FF7101830907C16102490162704791
:103B7000638A010000C0FF0F064941F6A260088079
:103B800005480168054A01F4E06111430160BFF393
:103B90004F8FFEE7442C01400CED00E00400FA05D5
:103BA00038B501210D2000F09FF94FF4E060ADF829
:103BB000000018248DF8034003258DF80250694653
:103BC0000D48FEF7FFFA4FF46040ADF800008DF8A5
:103BD00003400A4C8DF8025069462046FEF7F2FA7F
:103BE000A014ADF8000048208DF803006946204677
:103BF000FEF7E8FA38BD000000080140000C014063
:103C0000F0B50121CE028DB0304600F06DF95A4F6B
:103C1000384601F033FB08A801F05CFD4FF4586012
:103C2000ADF824000024ADF820402020ADF822009B
:103C3000ADF8264008A9384601F0FEFC00213846C0
:103C400001F051FD4FF6FF71384601F056FD01229B
:103C50000021384601F0E2FC0121384601F0CAFAA1
:103C600004A801F0E2FAADF810607010ADF812008F
:103C7000ADF81440A220ADF816007000ADF81800A1
:103C8000ADF81A40ADF81C4004A9384601F0BCFA62
:103C90006020ADF80000ADF80440ADF80840ADF884
:103CA0000C40ADF80240ADF80640ADF80A40ADF862
:103CB0000E406946384601F0A1FB6946384601F0DE
:103CC000E3FB6946384601F029FC7020ADF800009E
:103CD0000125ADF8045040F61450ADF80600ADF8DB
:103CE0000840ADF80C40ADF80250ADF80A40ADF810
:103CF0000E406946384601F055FC0121384601F076
:103D00009DFA0821384601F0B9FB3146384601F0EA
:103D1000FBFB0821384601F03FFC3146384601F0F4
:103D200073FC7021384601F07CFC18208DF82C00C3
:103D30008DF82D408DF82E408DF82F500BA8FFF7F1
:103D400091FD0D480C30018841F0800101800A4846
:103D50001430018841F001010180001F048001211D
:103D6000384601F075FA8DF828500121384601F0E7
:103D700079FA0DB0F0BD0000002C01407047000042
:103D800070B50189C1EB411101EB4101CA0B4281C0
:103D90000B49104603F0DCFC09480C38B0F90C2044
:103DA0000168B0F90E4001FB02F54368614303FB73
:103DB000145503FB0211AD138913C0E9055170BD01
:103DC000F409002040F213414160082181608621FE
:103DD000C1604FF4804101614942416100210162AB
:103DE000C16270470162704710B501884288891A24
:103DF00009B20183B1F5005F02DBA1F5804104E067
:103E000011F5005F02DC01F580410183B0F9182053
:103E100041685143C1618368846A5343C2681B127D
:103E2000624303EB2222036A1A44114402628A139A
:103E3000426241698A4203DB01698A4200DC114621
:103E40008A1AC0E90A21028E4FF40373594302EB28
:103E5000A13202860B4A1278082A04D10A4AD36E8C
:103E600003EBA131D166B0F93010B1F5804F02DD1E
:103E7000A1F5804103E0002902DA01F580410186C5
:103E800010BD0000F7060020240A0020034A5168F4
:103E900021F440410143516070470000001002408E
:103EA000044A0029516901D0014300E08143516176
:103EB0007047000000100240044A0029D16901D077
:103EC000014300E08143D1617047000000100240CF
:103ED000044A0029116901D0014300E081431161C6
:103EE0007047000000100240044A0029916901D087
:103EF000014300E0814391617047000000100240DF
:103F0000044A0029D16801D0014300E08143D16017
:103F1000704700000010024030B524494A6812F092
:103F20000C03234A03D0042B01D0082B26D00260B7
:103F30004A680F231F4C03EA1212A35C0268DA409E
:103F400042604B68072505EA1323E35C22FA03F37A
:103F500083604B6805EAD323E35CDA40C2604B68B8
:103F6000032403F4404104EA933303EB9161114BC2
:103F70001B1F595CB2FBF1F1016130BD4A680E4B69
:103F80001A404B68140103F4803303D5C2F3834213
:103F9000113202E0022404EB924213B14B689B03FE
:103FA00001D5064B00E0024B5A43C0E70010024027
:103FB00000127A000400002000003C0800093D00C7
:103FC0002DE9F041274CA61540212046FEF778F94F
:103FD000850080212046FEF773F945EA4005314609
:103FE0002046FEF76DF90543EDB240212046FEF76D
:103FF00067F9870080212046FEF762F947EA40070B
:1040000031462046FEF75CF90743F8B2A842DBD1FF
:1040100040212046FEF754F9870080212046FEF714
:104020004FF947EA400731462046FEF749F9074372
:10403000F8B2A842C8D140212046FEF741F98700D6
:1040400080212046FEF73CF947EA400731462046EA
:10405000FEF736F90743F8B2A842B5D12846BDE8C5
:10406000F08100000010014010B50268416802FBB9
:1040700002F301FB01330D4CA34211D91B0E0F3B80
:104080000B4C9BB212B234F8133009B25A43594365
:1040900042F38F3241F38F31C0E90221012102E066
:1040A000C0E902210021017410BD000040A45D0F91
:1040B000F08800082DE9F05FFD48FE4902880B8872
:1040C0009A1A92B20F2A76D309880180FA480246DA
:1040D0008189D2884B0703D48B0701D4CB0702D048
:1040E00042F4007201E022F40072C28083460807A5
:1040F00002D45846C90604D5BBF8061041F00101A8
:1041000002E0C18821F00101ABF80610EA48FDF792
:104110008BFEEA484FF48049B0F93A10494502DA7B
:10412000491C418701E0A0F83A90E54E41F6CC41A8
:10413000E44DB06C884203DDA86820F01000A86050
:10414000E14AE24FE2481188002411B1491E118072
:1041500008E0E98F41B1491EE987DE490A7822F07B
:1041600002020A70EC732DE0BBF806104B0419D460
:10417000BBF80C20D30615D4120713D40A0611D4A9
:104180008A060FD40A050DD44A0603D5D24A1278FE
:10419000120607D54A0705D4CA0503D40A0701D475
:1041A000C90609D5CD49EC73CD4A3C70CC83148047
:1041B00081F82A4007E07BE03978012903D10178B2
:1041C000062900D13C703978DFF8F8A2C54BAAF176
:1041D0002C0A4FF001080A2978D2DFE801F0FD69C6
:1041E0000569FCFB6977CDE4E87B09281AD0DFF884
:1041F000F8B202286CD0B5F8400010B39BF8680004
:1042000040F63A22012822D0C5F8D84085F8EA4085
:10421000CAF82040B5F9301001F21D50904226D85E
:10422000102325E0A2484430FEF736F9FDF776FE6C
:10423000716CCAF8281041F27C510920CAF8181094
:104240007AE1AA48018B2986A5F8408015E0A848A4
:10425000C5F8D80085F8EA80B5F9301001F21D5391
:10426000934201D8102300E02023102202E02023F3
:104270001022002000F0FAFA28869BF868309D4949
:10428000012B736C40F2DC504FF4927212D08342D7
:1042900004DA9648B0F90A00904212DBB5F84020E3
:1042A00040F6C410521C92B2A5F84020824208D2B7
:1042B000BDE8F09F8342FBDA8C48B0F90A009042D7
:1042C000F6DA3C7085F8EA404C83F1E7B1E0FFE7AD
:1042D000716CCAF828108AF807808748A5F8404012
:1042E00085F8EA40427F56465AB1C17F99B3C477F8
:1042F00080F81D40B5F93000484539DDA5F830900B
:10430000D6E708B27D4901F001FCA5F8E400A96AEE
:10431000814200DA084600B2B0829BF84D100029B5
:10432000B5F9301002D03623052201E0A3230A227A
:1043300000F09CFA2886B5F91601B5F914118842E7
:104340000ADA317901F10101C9B231710429D1D3FD
:104350003471401C02E007E003DD801EA5F8160161
:10436000C8E7A5F81611C5E740F266602886C1E7E0
:1043700000289DDA2C869BE76148D5F8DC10814245
:1043800002D2491CC5F8DC10E97B082903D1D5F815
:10439000DC10814203D33C70C5F8DC4088E7BDE8FF
:1043A000F05F02F01BBCE87B092801D02C8631E1CC
:1043B000DAF81C005746401CCAF81C0002280DDD24
:1043C000388D012301B2388B052200B200F04EFA7D
:1043D000FC6102E011E00CE013E0B8623448398D72
:1043E00044300180B6F844104180FEF76DF828860D
:1043F0005EE7BDE8F05F04F03DB91878092856D0B3
:1044000056E740490A78521CD2B20A70C82A10D323
:104410003D4A92F800C0BCF1010F0AD114700C7033
:10442000BBF80620394922F40062ABF8062081F877
:104430000080E97B891E08296ED2DFE801F006B210
:10444000EDFD056D8E04EDE632E7FDF773FF307884
:10445000400611D52E48807804280DD0706C822833
:104460000ADAB07A00F0030196F83D0000F003008C
:10447000814201D001F04AFD387806288ED086F8B6
:104480003F40B06C40F311011848C16221488903D4
:104490000162FDF743FD8AF80780B5F81401A5F81D
:1044A0001601706CA5F88240B0F5437F35E0B1E0AD
:1044B0002009002000070020100A00202405002009
:1044C00044010020A002002004070020F70600207D
:1044D000F8060020CE050020D8060020B4080020F1
:1044E000240000205C020020640C002068000020F2
:1044F0009AF9FFFF900900202C0C0020248C000862
:10450000C0D401001A0100201B010020140000206B
:1045100044040020900800209BE0A5F880900DDD69
:10452000A86840F48060A86096F8381005298BD1FF
:1045300040F01000A8606BE03870B9E6A96821F47B
:104540008061A96040F28A21884204DA307840060E
:1045500001D402F02FFAA868EAE7716CB1F5437F45
:1045600004DA0178062901D004706BE03C48017838
:1045700021F040010170FDF7D1FCA5F81691FDF77F
:10458000D9FE384810F8281F21F001010170364982
:10459000C5F8DC400C6235490C620821397044646E
:1045A00086E69BF80600C006C7D4706CB0F57A7F2B
:1045B00030DDFDF7BFFE3078400611D52C488078FD
:1045C00004280DD0706C82280ADAB07A96F83D1073
:1045D00000F0030001F00301884201D001F096FCD5
:1045E00086F83F40B6F84800288601B22C46494577
:1045F00001DDA4F83090FDF791FCA06840F48060E4
:10460000A06096F83810052997D140F01000A060FE
:10461000022091E73C704BE6716CB1F5437F02DA02
:1046200001780629A0D1BBF8061021F02001ABF8D3
:104630000610FDF77FFE00E001E004207CE7007833
:10464000062802D087F8008032E60920187005207D
:1046500072E707498C700470064880F8564089E676
:1046600006070020240A00206C0800209008002083
:10467000440400206800002030B585B001210420EA
:10468000FFF732FC4FF40040ADF8100048208DF8E1
:10469000130004A91848FDF795FD01210846FFF70E
:1046A0000BFC40F68C20ADF8040003240020ADF88C
:1046B0000040ADF80200ADF806004FF080456946B5
:1046C000284600F0B9FF1C208DF80C008DF80D4035
:1046D0008DF80E4001208DF80F0003A8FFF7C2F8F7
:1046E00001221146284600F081FE0121284600F0F3
:1046F000AFFD05B030BD000000080140704700006C
:104700002DE9F041304CE07800285AD1207800287B
:1047100057D0401E10F0FF00207052D14FF4967019
:10472000208272B6294F45F2AA50A7F872000020E5
:10473000FDF7D2FB264D13202860FDF7DFFBA8BB59
:104740003420E86002202861224E6E61286940F022
:1047500040002861FDF7D2FB40BB00211E4A0846FD
:104760005FEA255312F800C0BCF1FF0F00D0012111
:10477000401C80B29842F5D3C1B9C4E90676392607
:104780000127A06910F8011B10F8012BA061E06956
:1047900001EB022102886A612F6120F8021BE061AF
:1047A000FDF7ACFB10B9761EB6B2EAD20120FDF7D8
:1047B00093FB62B601F0FEFB0848816821F480415A
:1047C0008160BDE8F0810000F4060020640C002048
:1047D0000020024000FC000800FC0008A0020020AD
:1047E0001948016841F010010160016821F00301DE
:1047F0000160016841F002010160144841684160B4
:1048000041684160416841F480614160416821F440
:104810007C11416041680E4A11434160016841F0DA
:104820008071016001688901FCD5416821F00301B4
:104830004160416841F0020141604168C1F381017A
:104840000229FAD170470000002002400010024007
:104850000000280830B5044C039D6080A180E280F0
:104860002381658130BD0000040A00200A44824291
:1048700001DA10B27047C91A8142FBDD08B27047F5
:10488000F0B53E48DFF8F8E03E4CC17F467A056857
:1048900000233D4A3D484FF0010C802925D301F00B
:1048A0001F015EF821100D420146096802D041F453
:1048B000805101E021F480510160CF0411D48F04B4
:1048C0000FD5977AFF0705D05381277827F0020785
:1048D000277006E090F846709FB1012F14D080F841
:1048E00046300F0B67F34D310160802E25D306F063
:1048F0001F015EF821100D42016809D041F004014A
:1049000008E080F846C0ECE7022780F84670E8E748
:1049100021F0040101604D070BD44D0509D5957AAE
:10492000ED0706D05381257825F002052570C0F8E3
:1049300098308C0864F38A210160917AC90718D1F4
:10494000134991F86410012913D11249496C322995
:104950000DDC017849070AD50189090507D4D0F88B
:10496000981047F23054A14204D9A2F80AC0C0F806
:104970009830F0BD491CC0F89810F0BDD405002057
:1049800048910008CE050020100A0020A002002057
:10499000640C00204401002010B5FCF7E9F90F4831
:1049A000018821F0020101800C49183109880C4A64
:1049B000928E1144094A3432118008490C390A8810
:1049C00042F001020A80011D0A884FF6ED531A4099
:1049D0000A80018841F01201018010BD0C040040E2
:1049E0004404002006480188491C89B20180B1F5C1
:1049F0007A7F04D34188491C41800021018070479F
:104A0000180700200F4810B5016841F0010101604E
:104A100041680D4A1140416001680C4A1140016033
:104A2000016821F480210160416821F4FE014160A8
:104A30004FF41F018160FFF7D3FE05494FF000607E
:104A4000086010BD001002400000FFF8FFFFF6FEF6
:104A500008ED00E02DE9F0412F4D28884FF00004CB
:104A6000000629D5FCF7FEFA2C4A2D4807231778B3
:104A7000C8262C49012F22D02B4FB7F806C0BCF115
:104A8000000F3ED0B0F80CC04CF0080CA0F80CC0E1
:104A9000B0F806C02CF4006CA0F806C0886820F0BE
:104AA00004008860FC801370CE8700204FF496616C
:104AB000401C80B28842FBD32C80BDE8F0811B4FA4
:104AC00097F800C0BCF1010F0FD0BCF1020F11D05C
:104AD000B0F806C04CF4006CA0F806C0886840F03E
:104AE0000400886005203870DDE7B0F80CC04CF099
:104AF000080C03E0B0F80CC04CF0100CA0F80CC08F
:104B0000F0E70B4F3C70C78847F40067C7808868A0
:104B100040F004008860C6E7102C0140F706002032
:104B2000100A0020A002002020090020F806002022
:104B300015070020704700002DE9F0434FF080403A
:104B4000018A21F001010182AC48007800287CD163
:104B5000AB4FF87B002878D1AA48406C322874DC2F
:104B6000A9488068DFF8A4924104A94DB9F804006F
:104B70004FF0000403D4401CA9F8040028E10028E9
:104B800074D02978012611B1012912D017E14946C4
:104B9000B0F5BE7FFAD92E70CC718C71EC702C728E
:104BA000287A0A18401CC0B2147228720F28F7D352
:104BB00005E1B9F802204946824201D9EE7100E0D0
:104BC000EC7192488A7908300F2A15D2CB79082BDC
:104BD0000BD2C3F10708EB7912F800C003FA08F30F
:104BE00063441354CA79521CCA71CA79082A03D182
:104BF0008A79521C8A71CC7199F80610C8460F291F
:104C000073D10D21FCF798F9A881010A6970C0B22F
:104C1000A87088F8064098F816208A4265D198F85E
:104C20001510814261D198F80BC07A490323022202
:104C30007948BCF1000F10D0BCF1010F02D0BCF1DB
:104C4000020F14D080F86A2000E0CBE091F800C099
:104C50002CF00C0C0CF1080C0FE080F86A6091F855
:104C600000C02CF00C0C0CF1040C06E0A9E080F85C
:104C70006A3091F800C04CF00C0C81F800C098F834
:104C80000C10B6EB111F04D180F86E4087F8464037
:104C90000EE0B2EB111F04D180F86E6087F8466019
:104CA00006E0B3EB111F03D180F86E2087F8462091
:104CB0000B0717D001F00F01012901D0022915D0EF
:104CC00080F86C602C7198F80D102A7906FA02F3BE
:104CD0000B406B71082A44D2DFE802F00B12431933
:104CE000242F363D80F86C40ECE768E080F86C20BB
:104CF000E8E713B180F8704033E080F8706030E08E
:104D000013B180F850602CE080F8504029E023B1C6
:104D100080F8656087F8036123E080F8654087F8D4
:104D200003411EE023B187F8F54080F84D4018E0BC
:104D300087F8F56080F84D6013E013B180F8686083
:104D40000FE080F868400CE013B180F8666008E07E
:104D500080F8664005E013B180F8676001E080F8F4
:104D60006740521CD2B22A71082AAED398F80E10AE
:104D70002A4A8B0705D587F8F16080F86460568170
:104D800004E087F8F14080F864405481C90702D0FC
:104D900080F8294001E080F8296098F8111000F8A7
:104DA0006D1FC2781E48012A1ED001B3012921D0EF
:104DB0004FF48051A0F876101A493C200870A9F8E9
:104DC0000240A9F80440B9F80210491CA9F80210E1
:104DD000B9F80210B1F5FA7F04D940F2F511A9F83B
:104DE00002102C70BDE8F08344F21C71E2E74FF42E
:104DF0000051DFE741F25551DCE70000F7060020E3
:104E0000A002002044010020001001404C0C0020B2
:104E100090060020BC040020640C0020100A002032
:104E200024050020F40600202DE9F05FFDF782FA4A
:104E30008E4D2888A5F10406C0070AD0308820F0DE
:104E400008003080288820F00900288001F0B2FD99
:104E5000D9E02888DFF81892DFF81882864C80079E
:104E60001AD5B9F8001041F00101A9F80010B8F8FE
:104E70000000804914315030088028884FF6F951DD
:104E800008402880308840F004003080FFF798F810
:104E900084F83C00BDE8F09F2888784F40072888B8
:104EA00071D520F004002880FFF78AF894F83C10B0
:104EB0008142EFD1308820F004003080FDF712FCF1
:104EC0002078410605D594F84C1094F83B20914287
:104ED000E0D03978400621F00201397004D5FEF7A0
:104EE00025FB97F82F7004E094F83C00FDF774FA66
:104EF0000746DFF880B140F68C2A0BF1180B062F1D
:104F000047D294F83800B8423ED03846FDF7E8F969
:104F10002078C00716D094F83A0094F8391000F0C1
:104F20000302914206D0A17A00F0010001F00101D4
:104F3000884215D1FDF73EFBFBF766FFFDF766FCE7
:104F4000384689E0FDF736FBFBF75EFFFDF75EFCB8
:104F50003846FDF74FFB207840F00100207099E7BC
:104F6000288820F008002880206B810801EBD00001
:104F7000504515D2B8F800100844ABF8000030884E
:104F800040F0080003E00DE0308820F00800308099
:104F900080E7B9F8001041F00101A9F80010DFE73F
:104FA0005046E7E70007288831D520F00800288020
:104FB000308820F008003080FFF702F884F83C00C9
:104FC000FDF790FB387820F002003870207840061A
:104FD00004D5FEF7ABFA97F82F5004E094F83C00A4
:104FE000FDF7FAF90546062D08D294F83800A842D4
:104FF000B5D0FDF7DFFAFBF707FF2AE02048C188AC
:1050000041F04001C180BDE8F05FFDF7DFBBC006A5
:10501000288825D520F010002880308820F0100046
:10502000308097F838000C2802D2401C87F83800EE
:10503000387840F002003870FEF778FA97F82F5071
:10504000787884F8390094F83800A84287D0FDF7C2
:10505000B1FAFDF7DBFB2846BDE8F05FFDF7CABA01
:105060004EF2BE110840288014E7000010040040F2
:1050700000040040240400404401002044040020B7
:10508000100A00202DE9F04F514F85B0388820F0EC
:10509000010038804E480026103006804D4CDFF865
:1050A00038A14FF0010894F85C0042F63029C1079E
:1050B00074D072B64948816941F400718161816997
:1050C00041F4806181614FF40040FEF7DFFE444D02
:1050D00000212846FBF7F6FB00212846FBF7E8FBFA
:1050E000DFF800B100215846FBF7E2FB00213E4803
:1050F000FCF772FA2846FBF701FD5846FBF7FEFC69
:105100004FF46020CDE902068DF8056000968DF819
:1051100010808DF8048069462846FBF781FD012345
:105120001A460F212846FBF7CCFD01212846FBF744
:10513000BFFB00204946401C80B28842FBD3284672
:105140002E600121FBF7FCFD28688007FCD5244870
:105150004C30006894F85C1021F001012144A1F862
:105160005000FBF7B9FB62B6FEF7ECF847F690612A
:10517000AAF8001094F85C00401CC0B284F85C00EF
:105180000C2822D212491431A1F80080388840F04E
:105190000100388005B0BDE8F08FFFE7134920F02B
:1051A0000100085A12490880114945F6580008398B
:1051B00008800F4847F25801001F01800C49202049
:1051C0000C390880AAF80090D4E70320A070E1E72A
:1051D00000080040440400202C0800400010024059
:1051E000002401400028014008000240048D00080E
:1051F000202C01400029018802D041F0800101E00B
:1052000021F080010180704710B50A884B88CC8856
:105210001A438B8823431A430B891A434B89898984
:105220001A430A43A0F8442010BD002101804180A8
:105230008180C180018141818181704700298188FD
:1052400002D041F0010101E021F0010181807047AD
:105250000029018802D041F0010101E021F00101A3
:1052600001807047002930F8441F02D041F400410A
:1052700001E0C1F30E010180704700004B4910B5F9
:10528000884202D10121C41486E0B0F1804F09D0D8
:10529000474988420DD101210220FEF719FE002165
:1052A000022064E001210846FEF712FE00210120E1
:1052B0005DE04049884206D101210420FEF708FE46
:1052C0000021042053E03C49884206D101210820F6
:1052D000FEF7FEFD0021082049E03849884206D14A
:1052E00001211020FEF7F4FD002110203FE0344999
:1052F000884206D101212020FEF7EAFD002120206E
:1053000035E03049884202D10121441444E02E495D
:10531000884202D10121CC043EE02C49884202D1CE
:1053200001210C0538E02A49884202D101214C05AF
:1053300032E02849884206D101214020FEF7C8FD0D
:105340000021402013E02449884206D10121802019
:10535000FEF7BEFD0021802009E0204988420AD1E5
:10536000841501212046FEF7B3FD00212046BDE84B
:105370001040FEF7ADBD1A49884202D101210C044C
:105380000AE01849884202D101214C0404E0164980
:1053900088420AD101218C042046FEF7B1FD204647
:1053A000BDE810400021FEF7ABBD10BD002C014050
:1053B0000004004000080040000C004000100040C5
:1053C0000014004000340140004C014000500140F6
:1053D0000054014000180040001C00400020004024
:1053E000004001400044014000480140002A8289F9
:1053F00001D00A4300E08A438281704730B5028CB5
:1054000022F001020284028C8388048B22F00202C3
:1054100024F073050C882C430D8915434A882A43D0
:10542000114DA8420BD0114DA84208D0104DA842F2
:1054300005D0104DA84202D00F4DA8420DD122F048
:1054400008054A8923F440732A4322F004058A8818
:105450002A438D891D43CB892B4383800483C988CC
:105460008186028430BD0000002C014000340140E0
:10547000004001400044014000480140028B22F0FE
:1054800008020A430283704770B5028C22F01002B2
:105490000284028C8488038B0D8823F4E6464FF641
:1054A000FF7303EA052535430E8922F0200203EA43
:1054B000061616434A8803EA02123243104EB042DF
:1054C00002D0104EB04215D122F080064A8924F451
:1054D000406403EA0212324322F040068A8803EA5B
:1054E000021232438E8903EA86062643CC8903EAF8
:1054F0008404344384800583C9880187028470BD95
:10550000002C014000340140028B4FF6FF7322F45F
:10551000006203EA012111430183704770B5028CD8
:1055200022F480720284028C8488838B0D8823F09D
:1055300073031D4322F400730E894FF6FF7202EAD3
:1055400006261E434B8802EA03233343104EB04223
:1055500002D0104EB04215D123F400664B8924F4DA
:10556000405402EA0323334323F480668B8802EA23
:10557000032333438E8902EA06162643CC8902EAC6
:105580000414344384808583C9888187038470BD73
:10559000002C014000340140828B22F008020A43B3
:1055A0008283704770B5028C22F480520284048C8E
:1055B0008288838B0D8823F4E6464FF6FF7303EA57
:1055C0000525354324F400560C8903EA043434439A
:1055D0004E8803EA06362643094CA04202D0094C05
:1055E000A04205D122F480448A8903EA8212224330
:1055F00082808583C988A0F84010068470BD0000B1
:10560000002C014000340140828B4FF6FF7322F4DE
:10561000006203EA01211143818370470185828280
:105620007047828822F07002828082880A438280DA
:105630007047A0F84010704730B502881B4B1C4CD7
:1056400098420DD0A0420BD0B0F1804F08D0194D38
:10565000A84205D0184DA84202D0184DA84203D147
:1056600022F070054A882A43154DA84206D0154DF0
:10567000A84203D022F44075CA882A4302808A884F
:1056800082850A88028598420AD0A04208D00E4A34
:10569000904205D00D4A904202D00D4A904201D16D
:1056A000097A01860121818230BD0000002C014071
:1056B000003401400004004000080040000C00409D
:1056C0000010004000140040004001400044014030
:1056D000004801404FF6FF71818000210180C180A8
:1056E0004180017270470029018802D041F0020117
:1056F00001E021F00201018070470029018802D0F9
:1057000041F0040101E021F0040101807047000034
:10571000224810B590F82010026801F01F002049BF
:1057200051F820001F490242086802D040F480303E
:1057300001E020F4803008601B484FF000048079BD
:1057400041061A4827D41A4A01881388591A89B27F
:1057500001230F290BD3118801808168002900DC07
:105760004942042903DB13490978022905D0417F06
:10577000012906D01188418010BD4377C477118874
:10578000418041881288511A89B240F635429142CF
:10579000F2D3C37710BD447710BD0000D4050020BC
:1057A00048910008A0020020100A00202C0C0020C4
:1057B00000070020F70600202DE9F04FDFF8B8B110
:1057C0006A48DFF8AC91DFF8ACA190F80EC0BBF9E5
:1057D0001A70BBF91C60BBF91850BBF96C10BCF116
:1057E000070F48D2DFE80CF08D041A30485E7600CF
:1057F000D9F800208284DAF80020C284828CC38C1D
:10580000A7EB820212B2A6EB83034A431BB25943B1
:1058100042F3CF2241F3CF23D11870E0D9F8002012
:105820004284DAF80020C284428CA5EB820213B2D3
:10583000C28C4B43A6EB820212B243F3CF245143F6
:1058400041F3CF23E11814E0D9F80020C284DAF83C
:1058500000204284C28C438CA6EB820212B2A5EBDC
:1058600083031CB24A43614342F3CF2341F3CF2465
:10587000191949420AB244E0D9F800208284DAF8C2
:1058800000204284828C438CA7EB820212B2A5EBEB
:1058900083034A431BB2594342F3CF2241F3CF243F
:1058A000111914E0D9F800204284DAF8002082842B
:1058B000428C838CA5EB820212B2A7EB83034A438E
:1058C0001BB242F3CF24594341F3CF22A1184942DE
:1058D0000BB216E0D9F80020C284DAF800208284E6
:1058E000C28C838CA6EB820212B2A7EB83031CB29C
:1058F0004A4342F3CF23614341F3CF2299184942EF
:105900000CB2BBF91E50594605F21E56A64201DAEA
:10591000CE8306E0A5F21E55A54201DDCD8300E051
:10592000CC83B1F9204004F21E55954201DA0D8472
:1059300006E0A4F21E54944201DD0C8400E00A84C7
:10594000B1F9222002F21E549C4202DAABF8224046
:1059500008E0A2F21E529A4202DDABF8222001E0DA
:10596000ABF82230417B8173BDE8F08FA0020020AC
:105970003C2401403C280140240500202DE9F0474B
:1059800004465748584D002602785648022AB0F976
:10599000301004D0082A7DD0092A07D008E0C27B45
:1059A000022A02D1B0F8402032B1E18769812E810C
:1059B00084F83C60BDE8F0874C49DFF83481496ADF
:1059C0000F14E7808068410210D5B4F9020040F25C
:1059D000DA21884269DD40F26A4188423FDCA0F268
:1059E000DA20FAF71CFD0022424B4BE0C0F3C00165
:1059F000C0F30020DFF8009181420CD1D8F84400B8
:105A000040F2BA41884250DD40F66A11884226DCF5
:105A1000A0F2BA4032E039480078C0060CD5D8F878
:105A2000440041F2243188423FDD41F2D471884282
:105A300015DC00F6DC401FE0314890F870100129B9
:105A400003D090F86F0001282FD1B4F9020041F67D
:105A5000C811884229DD41F6786188420ADD0823B1
:105A6000B4F93E101A460020FEF700FFE087002838
:105A700019DB1BE000F5C760A0F50050FAF7CFFC7A
:105A800000224B46FAF737FC0E22FAF7A3FCFAF78E
:105A9000FDFC00E01FE000B2C0F5804078438013B9
:105AA000E087002F02DCE68700E0E787E08F154FF4
:105AB000E880D8F844107964A7F84C0000F076FB31
:105AC000B7F84E00688198F80A000028388F00D196
:105AD000404228816CE70C48B0F87000688166E7A6
:105AE000F7060020A0020020680000202405002006
:105AF000440100200000794000C09240D8060020F8
:105B0000640C0020B4080020240A00202DE9F04194
:105B1000B1F9025000232B241522854203DAB1F992
:105B20000000BDE8F081B1F9AE50854202DDB1F967
:105B3000AC00F6E701EB8205B5F90250854201DDC4
:105B4000134600E01446E21852085D1CAA42F1D147
:105B500001EB8206B6F90230834206DA36F9025CBE
:105B600036F9044C31F9221006E01D4631F9224085
:105B7000B6F90630B6F90410401B091BC617891187
:105B8000B60346EA90468703A1FB070CCA1702FB3F
:105B900007C201FB06215A1BD317FAF7C5FA000A00
:105BA00040EA0160001900B2B0F5804FB9DB43F65E
:105BB000FF70B6E770B5134C40F2244529462046E5
:105BC00000F03EF800281BD0204600F0C7F8294618
:105BD000204600F01DF80C4C00212046FBF7FCFC91
:105BE0002046FBF777FDC0F164000849C0B20428E5
:105BF000087201D900F046F9BDE87040FBF7B0BD6E
:105C000070BD0000003801405800024060060020CE
:105C10000A0A01219140C943018070470029818906
:105C200002D041F4005101E021F40051818170471C
:105C3000002A828A01D00A4300E08A4382827047A8
:105C400030B501F01F0201240025C1F3421304FA0C
:105C500002F2012B0FD0022B0FD0838A4FEA1121C1
:105C60000088134204FA01F400EA040001D000B1F4
:105C70000125284630BD8389F0E7038AEEE710B599
:105C8000C1F3421301F01F040121A140012B07D0F1
:105C9000022B07D01430002A026805D00A4304E022
:105CA0000C30F8E71030F6E78A43026010BD0000C0
:105CB00030B50446008A85B00D464CF6FF710840A9
:105CC000E98801432182A1894EF6F3100140A8889A
:105CD0002A8910436A890A431043A081A08A4FF69B
:105CE000FF410840A9890143A1826846FEF714F9E3
:105CF0001948844201D1039800E00298A18909045F
:105D000000EBC00101EB0010296801D5490000E05B
:105D10008900B0FBF1F06422B0FBF2F109010B093C
:105D20006FF018056B4300EB8300A3891D044FF04F
:105D3000320306D503EBC000B0FBF2F000F0070021
:105D400005E003EB0010B0FBF2F000F00F00084399
:105D5000208105B030BD0000003801408088C0F3CC
:105D600008007047F8B501210920FEF7BDF80121B0
:105D70008803FEF7B9F810258DF803502020ADF800
:105D800000001A4E03248DF8024069463046FCF7A5
:105D900019FA16490C31086820F020000860182014
:105DA0008DF803004020ADF800008DF802406946F0
:105DB0003046FCF707FA48208DF803008020ADF844
:105DC000000069463046FCF7FDF98DF803502801C4
:105DD000ADF800008DF8024069463046FCF7F2F954
:105DE00001210420FCF740FAF8BD0000000C01403E
:105DF00030B585B0FFF7B6FF00244FF4E1300090D6
:105E0000ADF808400C201D4DADF80440ADF80A0077
:105E1000ADF80640ADF80C4069462846FFF748FF4C
:105E200025208DF8100004208DF811008DF8124007
:105E300001208DF8130004A8FDF714FD012240F2A3
:105E400024412846FFF71BFF01212846FFF7E6FE05
:105E5000FBF7B0FC012280212846FFF7E9FE012272
:105E600040212846FFF7E4FE012202210448FBF707
:105E700045FCFBF79FFC05B030BD00000038014039
:105E80004400024070B51D4D00242878432834D1C9
:105E90006878462831D1A878502807D0512805D0F5
:105EA000812803D0892801D0212826D1144E707171
:105EB000E9787172A81C891CFBF776F8B072717AC8
:105EC000294409793182884217D106F10E00017800
:105ED00041F0020101700B48016841F020010160AE
:105EE000317A0948002204E02B5D03552A55641CD1
:105EF000E4B28C42F8D38078707170BD8C070020BA
:105F0000600600200C0C0140960B002070B51D208F
:105F1000FDF787FCFDF70AFB1D20FDF798FC1548EF
:105F200090F82F10144D0623144C85F8381090F873
:105F30003B1095F83B201143012A04D0022A07D0D8
:105F4000042A0AD010E0827A8A420DD0007B09E050
:105F5000027D8A4208D0807D04E0827F8A4203D09D
:105F600090F82000884200D12370002085F840007E
:105F700070BD00004404002044010020F70600200A
:105F80000B4800214180A0F1B0018A898280CB8931
:105F90001A44C2800B8A1A4402814B8A1A444281F5
:105FA000898A1144818143F6FF71C18170470000E5
:105FB000F4010020084940F61C72B1F90C0090422F
:105FC00002DA00F59F7005E041F2E302904201DD44
:105FD000A0F59F70C88170476800002038B513484D
:105FE000C16941F00401C1611E208DF8000002204A
:105FF0008DF801008DF8020001248DF803406846F9
:10600000FDF730FC0A4984200880094947F6906072
:106010002C3108800020091F0880054914310C80AC
:10602000091F0880081F048038BD000000100240CE
:106030000008004030B420491E4A45788B7A11464A
:1060400092F83B4091F83910AC4218D14BB103792A
:10605000994202D04379994201D140791AE080797E
:1060600009E08379994202D0C479A14202D182F831
:106070002F3011E0407982F82F0030BC7047C5788E
:10608000AC42FAD16BB1C379994202D0037A9942FA
:1060900005D1007A82F82F0030BCFEF77DBC407A33
:1060A000E9E7437A9942E2D00479A142DFD0007A4D
:1060B000E1E700004404002044010020FEE7000066
:1060C0002DE9F0470446007F012868D13548E18872
:1060D0000288511A89B2072916D30088E080B4F9E2
:1060E000000044F2DD414843401346F6D96148437D
:1060F0008013A060401000B2A0814FF08051B1FB2E
:10610000F0F0FAF787F92061B4F90C6096B1B4F9B0
:1061100002104DF6B05048430014A082B4F9047048
:106120004DF6B05207FB02F24FEA2245E58204D455
:10613000024603E00020E08330E0424212B22283B4
:10614000002D01DB2B4600E06B421BB2DFF85890BC
:10615000638398464FF4804AB24208DAFAF751F95D
:106160002169FAF724F8FAF778F9801304E0002996
:1061700001DA484600E05046E083B04509DA284697
:10618000FAF73FF92169FAF712F8FAF766F980137E
:1061900004E0002F01DA484600E050462084BDE8C4
:1061A000F08700000007002000C0FFFF10B528485E
:1061B000294C01782748022905D1C17B022902D147
:1061C000B0F8401029B1008EA4F84E0000202087BE
:1061D00010BD90F8462020482049022AB0F844001B
:1061E000097800B2C1F3810103D0012A0CD01C4907
:1061F00013E0012904D0022904D019496C390CE0BC
:1062000018490AE0184908E0012904D002291CD0E5
:1062100015496C3101E013496C31FBF72DFE0E4935
:10622000A4F8400080B2483101F092FAB4F94C0071
:10623000B4F94A2041425143891324F8381FB4F974
:10624000101048438013E08210BD07496C39E4E721
:10625000F7060020A0020020B4080020BC040020A3
:106260009A8B000812890008568A0008034800210A
:1062700080F82A10C183018770470000B40800200D
:1062800010B504000B462D4AC3F1000028D5644226
:10629000002B12DAA04207DA214600F027FA32F882
:1062A0001000C0F5404041E00146204600F01EFAD3
:1062B00032F8100000F5004038E0A34208DA214629
:1062C000184600F013FA32F8100000F540402DE0B7
:1062D000204600F00BFA32F81000C0F5803025E0BF
:1062E000002B12DAA04207DA214600F0FFF932F85B
:1062F000100000F5804019E00146204600F0F6F954
:1063000032F81000C0F5004010E0A34208DA214640
:10631000184600F0EBF932F81000C0F5804005E0B7
:1063200053B1204600F0E2F932F81000B0F5004F0A
:1063300001DDA0F5803010BD002010BD108D0008DB
:1063400040438013494300EBA13000220302002B9D
:1063500014DDB3F5001F01DC802001E04FF4005094
:1063600093FBF0F1014401EBD1714910814206D059
:10637000521CD2B20846062AF2D300E00021C8001F
:1063800000B2704702E008C8121F08C1002AFAD103
:1063900070477047002001E001C1121F002AFBD1A5
:1063A000704700002DE9F047A44CA54821880288D9
:1063B000511A89B20F297DD30088A4F13C052080B1
:1063C000288F08B1401E28872B789E4AC3F381008E
:1063D00001281DD0022820D0D18B98489A4FDFF891
:1063E0006C92407E0026B1F5926F1DD8142819D307
:1063F00078206076F88840F01000F88040F26660FF
:10640000A88123F001002870D67389F8006015E098
:10641000D08B00EB4000C00302E0D08B8C49484396
:10642000010CDAE7401C04E0B1F5DB6F06D310B1D4
:10643000401E607602E043F001002870B5F90200CA
:10644000B5F914304143C3EBC303C1F38F31C3F338
:10645000D10303EB510109B2A9829046D28B4FF0D0
:1064600080535043B5F91620C0F38F30C2EBC202FF
:10647000C2F3D10202EB500000B2E882AA6A4243A2
:106480001213EA6293FBF2F22A63724A1080A26846
:106490000A44A260E1680144E160207C401CC0B273
:1064A0002074072806D942F3CF002883C9106983D6
:1064B000E66000E0BFE0A66041F6C80126748842AD
:1064C00004DD298B644AB2FBF1F1E981C11789032C
:1064D00041EA9041800342F69B420023F9F724FEF3
:1064E000A88456482A78A0F13C005C49B0F906001F
:1064F000930700FB01F14FEA2141C2F3810215D558
:10650000012A07D0022A0BD04FF2685141430914E7
:10651000A18011E049F68C4250430014A0801FE096
:106520004CF6183141430914A18025E0012A0DD011
:10653000022A17D0A0806984494948430014E083A7
:10654000FBF7BAFA47480088C0B143E04AF65C322C
:1065500042431214A2804BF62C225043001468844C
:10656000E183EDE74DF2AC5141430914A1804EF2B5
:106570007C414143091469843B49DEE795F82000DA
:1065800000BB88F80F6089F80060B5F91A00A0F523
:106590000C519F39B1F56E7F18D8617FF42912D95B
:1065A0003249E8802E4AA1F8460050430014A880E2
:1065B000A1F84400FF2085F8200081F828002C492C
:1065C0003C20087006E0491C617703E0607F08B159
:1065D000401E6077B5F91A10B4F91E0081420EDD35
:1065E000A07E7D2809D9F88840F00800F88021486D
:1065F000017821F0020101700EE0401C06E0A0F2DB
:106600003D10814208DAA07E10B1401EA07603E062
:10661000F88820F00800F880B5F91810606908447F
:106620006061217E491CC9B221761F2903D940111E
:10663000A88366612676BDE8F0870000F804002094
:1066400000070020A0020020100A0020F70600200A
:1066500030330100C409002074E8260BCC0E010081
:106660004885010002070020D0450100640C00208D
:10667000F4060020CE050020024941F68B308862E6
:1066800070470000BC04002070B5164C0625207829
:10669000062825D2DFE800F003080E141A2112485C
:1066A000FAF7C0FC012016E00F48801DFAF7BAFC8B
:1066B000022010E00C480C30FAF7B4FC03200AE08A
:1066C00009481230FAF7AEFC042004E006481830FE
:1066D000FAF7A8FC0520207070BDFAF7C3FC2570FE
:1066E000257070BDF8060020068C0008090A05D048
:1066F000B0FBF1F0FF2800D9FF2070470020704761
:10670000D0E90021C368521A5A4301EBA2318160DB
:1067100041607047B0F90020B0F90210B0F90630BE
:10672000521A5A4301EBA231818041807047000028
:10673000F0B54F4C20884F49504E514B8A8A801AF1
:1067400082B24D480F2A057801F1540032D32288D5
:106750008A82197A5FEA017C0146B1F9021001F1DF
:10676000020217B2A1F1020212B20BD5022D01D022
:1067700044490FE0DFF810C1BCF900C0614513DCEB
:1067800017DB13E0022D15D1D6F844C0BCF5FA5F33
:1067900003DC3E49098841800CE0DFF8F4C0BCF915
:1067A00000C0614505DB01DD428003E0A0F802C0C6
:1067B00000E04780018F2288A2EB010189B29C2969
:1067C00041D321880187996A0022B1F5804F2CDBE3
:1067D000B16CB1F5405F28DD2E4940F26664B1F935
:1067E0001010A14211DD43F69914A14202DB40F2E0
:1067F000333108E040F23334A1F26661614343F281
:10680000333491FBF4F1818700E082872249B3F8A9
:1068100006410978C1F381011CB1818F01F21E513B
:1068200019E093F84630022B0ED08287022D00D05B
:106830008287B0F95410B0F93C2001F1140393425F
:106840000BDAA0F85430F0BD012901D00229E4D1BF
:10685000818F01F233318187E8E702F11403994215
:1068600003DD1439A0F85410F0BDA0F85420F0BD99
:106870000007002014000020F7060020440100203B
:10688000A0020020BA040020B8040020B6040020B2
:10689000B404002024050020BC0400202DE9FC41A4
:1068A00001210220FDF708FB01211920FDF71CFB47
:1068B00001213C48FBF7D8FC4027ADF800700324C9
:1068C0008DF802400420384D8DF8030069462846B3
:1068D000FBF778FCE001ADF800008DF802401C20C9
:1068E0008DF8030069462846FBF76CFC4FF4E07115
:1068F0002846FBF7EEFCA815ADF800008DF8024025
:1069000010208DF8030069462848FBF75BFC4FF424
:10691000A060FCF7D9FF1D208DF8040001268DF83A
:10692000056000258DF806508DF8076001A8FCF77A
:1069300099FF1F498C2008801D494FF6FA702C31B1
:1069400008806E20091F08801948143006801848F6
:1069500008300780164920310D80154AD020121DBD
:106960001080134A45F2F300183210800A1F45F2D6
:10697000500010800E4A4FF6FF7038321080121D02
:106980001080121D108041F21B10088000F012F8D8
:10699000FBF71CFF064810300580001F0480BDE88F
:1069A000FC810000000C1A0000100140000C0140A6
:1069B0000004004070B51D20FCF728FF2A4D40213F
:1069C0002846FBF77DFC840080212846FBF778FCF5
:1069D00044EA4004A9152846FBF772FC0443E0B2E0
:1069E000224C84F83C00FBF7F7FC0546052805D946
:1069F0001F48C18841F04001C18001E084F838504F
:106A00001C48007A000703D594F838001A490D5C39
:106A10004FF6FA702063E062A06260622062E0617B
:106A2000A0611648606300206064A06484F83F00A1
:106A300084F84000FBF77EFCA07AFF2811D00220EA
:106A400084F83D000E48008820662846FCF720F9AF
:106A5000207820F001002070BDE870401D20FCF778
:106A6000EBBE0120ECE700000010014044010020D3
:106A7000100A0020A002002014950008DCFF050089
:106A8000240400402DE9F0434E484F4902880B880A
:106A90009A1A92B20F2A69D3098801804B49098B4F
:106AA000027D00EB42029180017D491CC9B2017553
:106AB00008295BD3002404752246017D00EB4103C5
:106AC000491CB3F90430C9B202EB630212B201757A
:106AD0000829F2D33E4904753E4B4A8044800E7823
:106AE0009D895FEAC67C40F638694FF0030714D0F1
:106AF000A2F22B5C42F6E858C44520D3A1F1020C67
:106B000026F00204ACF8002047750C7040F22B54BC
:106B1000A24211DA45F004021EE046F001060E70B2
:106B20004A4507DD45F001029A8126F002020A700B
:106B3000477519E0447517E045F002020CE04A453C
:106B40000CDA8775427D12B1521E42750CE046F098
:106B500002020A7025F007029A8105E0B30703D507
:106B6000837D2BB15B1E837540888880BDE8F083F0
:106B700042F6AA239A4222DAB1F904302BB941F243
:106B8000CD05AA4201DA4480EEE7134C920302EBF2
:106B9000843241F67244B2FBF4F214B240F233355F
:106BA00002464480AC4200DA5580B2F90240E41A51
:106BB00004F5A374B4F5237FD6D84380D4E74FF40B
:106BC0008043FAE7980A002000070020A002002076
:106BD000CE050020100A0020C8F1FFFF2DE9F0418A
:106BE0006C4CDFF8B4E14FF0000594F82810C807AA
:106BF00006D094F92C104B42002956DD0E4655E084
:106C0000664884F82B50E586654A90F8380084F889
:106C100034001586CEF80450CEF80850614E40F28C
:106C20006663CEF80C50A4F8703036F810005E4E53
:106C3000768830444FF6FF7606EA800024F8240B6D
:106C40004FF080602060A320208460845810A084CE
:106C5000E38440F699102085580060854FF48050F9
:106C6000A08541F23330E08541F26660208641F62E
:106C70009910608641F6CC40A0864FF40050E08623
:106C800042F23330208742F26660608742F6991004
:106C9000A08742F6CC40E08782F89D5041F0010089
:106CA000207184F84450BDE8F0811E4694F92B0011
:106CB0004242002801DD074600E01746F61B012E80
:106CC0000BD0002800DB02465FFA82F684F82C0025
:106CD00094F84300012805D041E0002900DA194664
:106CE000CEB2F3E794F92D305942002B01DB184660
:106CF00000E0084694F92E20C7B25042002A01DB7A
:106D0000944600E08446BC4508DD002A00DA0246CD
:106D1000D7B2002B00DA0B46D8B207E0002B00DA1E
:106D20000B46DFB2002A00DB1046C0B204EB400085
:106D3000B0F9441004EB470030F9442F11444910D6
:106D4000018084F8435084F8325084F8315084F83C
:106D5000305084F82F5084F82E5084F82D5004EBD6
:106D600046007546B0F94400E086BEF80410C8231A
:106D700009B26422FDF77AFD6860E968401AA968E3
:106D80000844A860B5F900104843C013E860A4F8AF
:106D9000700088E7240A0020BC0500204401002080
:106DA000A002002026950008680000202DE9F0418F
:106DB0005F4C94F82800C00779D05E4894F83410EE
:106DC000002690F838005C4D814271D05B4AA4F8EF
:106DD00066605B4F535C2246834292F92B2002D0BF
:106DE0007B5C83420FD1521C52B284F82B20795C19
:106DF000814202D1521C84F82B2094F92B100F29C8
:106E00001BDD0F2117E04F4B5F5C4F4B874202D0D9
:106E10005F5C874211D1521E52B284F82B20595C1C
:106E2000814202D1521E84F82B2094F92B206FF05E
:106E30000E018A4201DA84F82B103D4994F8333070
:106E40002D3194F82B205A5494F83310491CC9B2B0
:106E500084F83310062901D384F8336094F92D2087
:106E600094F92F108A4211D194F9312091420DD119
:106E700094F92E2094F930108A4207D194F93220E7
:106E8000914203D1012184F8431001E084F843606A
:106E9000284984F8340094F92B300978012B0DDD52
:106EA000254A4F07926804D542F0080203E03CE00F
:106EB00015E022F00802AA6084F82900B3F1FF3F30
:106EC0000ADA4907A96802D521F0080101E041F07A
:106ED0000801A96084F82900FBF72CFA11E094F866
:106EE000430001280DD1B4F8660043F60951401C57
:106EF00080B2A4F86600884203D9A4F8666084F8DA
:106F00004360E87B082810D0B5F9301051234122A6
:106F10000020FDF7ABFC2886002806D10B48067040
:106F200014F8280F20F001002070BDE8F081000067
:106F3000240A002044010020A00200200895000837
:106F40000E9500081A95000820950008F706002005
:106F500030B52049204AB1F86A301088C01A80B292
:106F60000F2836D31088A1F86A001C4D00204FF07E
:106F700000432A5C940903D00124B4EB921F24D16E
:106F8000D20622D0164A52F820201268134C12342E
:106F900034F81040224201EB000494F9722008D02A
:106FA0000A2A04DB0A6823FA00F4224308E0521C90
:106FB00009E012F10A0F05DC0A6823FA00F4A24383
:106FC0000A6002E0521E84F87220401CC0B21128F0
:106FD000CFD330BDD4050020000700201491000855
:106FE000149200082DE9F00779497A480A89038844
:106FF0009A1A92B2082A74D300880881A1F12C0051
:1070000042890AB1521E4281734A92F82820802A8E
:1070100067D302F03F020A70C2890AB1521EC281D0
:10702000B1F90620902A0CDB8A46FF2A09D0814656
:10703000C089002855D1694800230078092805D067
:1070400005E0BDE8F007624800F092B90823644A01
:1070500092F8EA500DB143F004036248817AC907FF
:1070600001D043F00203D2F808C05FEA0C5101D509
:1070700043F00103176800215B4EFC0302D596F82C
:10708000654004B18021C4885FEA446801D541F0BD
:1070900040015FEA845801D541F020015FEAC478DD
:1070A00001D041F01001007A400701D541F00801FC
:1070B0004E480078C00701D041F00401A00601D578
:1070C00041F001010020012D00D1082096F87050F8
:1070D00085B992F84620022A04D0012A05D03AB197
:1070E00008E072E040F0030004E040F0020001E03C
:1070F00040F001007A0701D440F02000CCF3C00238
:107100000025CCF3002C624502D13A0700D40425B7
:1071100096F86F20012A01D145F00105344A002775
:10712000BC4612783E46C2F38102012A04D0022AEC
:1071300004D0032A04D004E0022602E0042600E082
:1071400010262C4A64060ED5214C1C3424782406C3
:1071500009D51478640606D4274A40F6CC44926DCB
:107160006243140C05E0B2F8AE2040F69914624375
:10717000940B4FF008088AF80A804FF061088AF8EB
:107180000B808AF80C308AF80D108AF80E008AF805
:107190000F508AF81070270A4B4083F06901414074
:1071A00069408AF8117079408AF81240614052466D
:1071B0008AF813C071408AF8146051754FF4C87191
:1071C000A9F80E10FF20AAF80600BDE8F0077047E6
:1071D000BC06002000070020D4050020F706002090
:1071E000A0020020100A0020640C002008090020E2
:1071F000BC04002044010020F00700204C488169B5
:1072000041F0FC0181614FF4A060FCF75DFBFBF7EE
:107210006BFBFCF7C5FCF9F7C9FCFCF7B3FAFDF70B
:107220002BFAFFF73BFBFCF7F3F9FFF7C3FBFBF788
:10723000CDFA404D4FF40050A5F81601FEF7D8FDE9
:1072400000214FF4FA5340F2EE220020401C80B29D
:107250009842FBD3491C89B29142F6D336480026A6
:1072600080F87260F9F738FBF9F7D2FFFCF7C8FC39
:10727000F9F7A6FEFEF7B2FE102230493048F8F7C3
:1072800084FF304C314FE08820F04000E0802E48F1
:10729000017821F020010170FA20F8814FF49670F6
:1072A000E887FFF7E9F92A492A48FCF71FFC2A4832
:1072B000FCF748FC2948416A88472948416B8847C0
:1072C000FEF7D4FF27494220C8802749C8603E7195
:1072D000E088E0812089208260896082FAF7EAFEF6
:1072E000FAF74CFEFFF75EF8FFF7CCFB00F0F8F979
:1072F000FFF72EFE01F082F8FEF70AFAFAF7ACFC6F
:10730000FBF7E4FCFFF714FAFCF7D4FEFBF706F9F1
:10731000FBF738F900F07AF8FFF764FE1348FAF744
:1073200093FA00F06FFAFDF7EBF9FAF7F7FBCFE706
:1073300000100240A002002024050020640C002060
:1073400014060020100A002044010020F40600204A
:10735000900800206C080020000400203C00002061
:10736000D80000201C0700203004002090090020D5
:10737000F0B523490278B0F9064000231F4E31F8DA
:107380001210FF2C18D0B0F904701E4DBC4231DA37
:1073900000EBE40704F00704BF7AA7408478FFB24B
:1073A0003CB190F801C0ACF1010C64451FDA3C0619
:1073B0001DD455F822200DE056F822201160124904
:1073C0008A79521CD2B28A71022A02D38370C38096
:1073D0008B71F0BD11608178491CC9B2817042780F
:1073E0009142F6D38370C188491CC180F0BD56F824
:1073F0002220EFE755F822201160F4E7F49200080C
:10740000269100089C92000890060020F0B5614883
:107410006149B0F86C200B889A1A92B29C2A7BD3EF
:107420000988A0F86C105D495D4F91F82A1001F0B1
:10743000070297F84610022A00D1491E594C80F8DD
:107440003E104FF00203E2884FF00001550401D5D1
:10745000012236E0A489E50601D5062231E02507A0
:1074600001D508222DE0550603D44F4D2D78AD06E9
:1074700001D5042225E0150501D5072221E01506D6
:1074800001D50A221DE0950601D50C2219E0150749
:1074900001D50B2215E0550701D4D50501D51022E1
:1074A0000FE0D50601D505220BE0650703D4A5073B
:1074B00001D4E40702D080F86E3007E0920403D5CF
:1074C000032280F86E2001E080F86E10374A384CB5
:1074D00092F820E0324A251FD2F808C02D4AB2F8AF
:1074E0007060721C92B2BEF1000F0DD02CF4000C33
:1074F000C7F808C090F86E70B7B11E2F1AD090F878
:107500006F200AB325E007E04CF40006BE60A0F847
:1075100070200A2A01D22360F0BD142A01D22B6008
:10752000F0BDA0F87010F0BD2B60A0F8701080F8CE
:107530006F10F0BD642E04D2A0F87020322AEED372
:10754000E9E7A0F87010EAE77F1C80F86F70A0F8F8
:10755000701090F86F20012A10D0002AE9D0B0F8FE
:107560007060761CB6B2A0F870601E2ED7D3236070
:107570003C2EDED9521E80F86F20D2E7B0F8702082
:10758000521C92B2A0F870202360C82AD1D980F88A
:107590006F10C6E7D405002000070020640C00200F
:1075A000A0020020100A002044010020BC0400209A
:1075B000141C0140F0B54248B0F84810491C89B28B
:1075C000A0F8481002297AD33E490024A0F8484088
:1075D0000A783D4B042A57D04FF48041082A0BD03B
:1075E000A0F10C02B2F900208A4200DA1146B3F988
:1075F00080208A4200DA1146344A92698A4200DACF
:1076000011B2418282881D8AC2EB8502304D12B2CE
:107610002D78C5F381062A4D42F2AA467243B5F988
:10762000765092126A431213C26086681546C6EB02
:10763000C60642F3D102F60202EBA6328260C66CA5
:107640001644C664B0F850707F1CBFB2A0F85070EA
:10765000B7F5806F04D3B6120682A0F85040C46418
:10766000891A1C4EC26A724340F255564E4302EBD1
:107670004602466A32444262B3F93030B2EB034FFD
:1076800006DD1A04426206E01349B1F90410B3E7BB
:10769000002A00DA4462C162104990F83D2091F856
:1076A00038108A420BD080F83D10B0F84210A0F894
:1076B0004410B0F84010A0F84210A0F84050F0BDBF
:1076C00024050020F7060020A0020020FC0B00206B
:1076D000BC040020C3F5FFFF180C0020440100206B
:1076E00017481849B0F85A200B889A1A92B20F2AF4
:1076F00025D30988A0F85A10134941F6515391F83F
:107700004D10CA0701464FF48042B1F900105943A9
:107710008913A0F86C100D490B78A0F10C01022B15
:1077200006D1B1F90030934202DA1B1D0B8000E054
:107730000A800021A0F8601020F85C1F428070478A
:107740002405002000070020640C0020F70600201C
:107750004FF6FF7202EA800210F4404315480ED043
:10776000B3F5804F14D0B3F5004F4FEA122216D074
:10777000C2F5807330F813305B424B8005E0120A8B
:1077800030F812304B80C2F5807230F812000FE0F2
:10779000120AC2F5807330F813304B8005E030F8E0
:1077A0001230C2F580725B424B8030F812004042CA
:1077B00008807047108F0008104A518A908AD28A38
:1077C00016384639A2F1110200D54942002A00DAE2
:1077D00052421144002800DA40420844084943F666
:1077E000284300B2B1F936205A43921340F2D733FE
:1077F000584302EBA030C88670470000A00200206A
:1078000024050020F0B5904990480A8903889A1A07
:1078100092B23E2A1ED30088088101F138004FF44D
:10782000FA63428A9A4202D2521C428200E04382A8
:10783000874A92F82220802A0CD302F03F020A7075
:10784000B1F90620402A06DBFF2A04D0C2883AB1EB
:10785000521EC280F0BDBDE8F0407B48FFF788BDF6
:10786000428A9A42F6D307784FF0010E3A074FF05A
:10787000FF055BD5847A40F2DC52630708D444F0FC
:1078800004038372C28081F80BE081F80AE04CE0C7
:107890004378072B05D0032B03D0052B01D0062BF3
:1078A00007D1660605D444F040038372C2800522E6
:1078B00039E0654A5FEA437C02F138024FF42076F2
:1078C000127A0DD55FEAC26C0AD45FEA446C07D421
:1078D00042F0100202723A0628D4C680192222E031
:1078E000DF0709D0970707D4670605D442F00202E4
:1078F0000272C680042216E09F0709D5170707D435
:10790000670605D442F008020272C68003220AE02C
:107910001B070BD5530709D4630607D442F00402B2
:107920000272C6800B22CA728A72CD80494AB2F9AD
:107930002230B2F91A7003F23D140022A74200DB94
:107940000276414E444C06F13806A479B6895FEAC6
:10795000C46C06F101064FF4C874B6B213D5868123
:10796000B6F57A7F05D9017A21F080010172828112
:10797000F0BD037A1E06FBD4828143F080020272BE
:10798000C480112035E09F4216DA037E052B13D206
:107990008681B6F5487F04D98281027A22F04002BE
:1079A0000272027A5606E3D45B1C037642F0400270
:1079B0000272C48002201CE0284B1C89C4F3C0065C
:1079C000C4F3002740F2EE24BE4216D11E783607DB
:1079D00013D4427E012ACBD1428BB2F5167F02D25C
:1079E000521C4283F0BD827A42F002028272C4804D
:1079F0000F20C8728872CD80F0BD93F80D714FF4DE
:107A00000046012F18D1164F41F6583C7F6C674550
:107A100012DD83F80CE1134B1E60C38AA34202D22D
:107A20005B1CC382F0BD4FF4FA73C3801C23CB727E
:107A30008B72CD80C282F0BDC2820A4883F80C21CD
:107A4000001F0660F0BD0000A00600200007002017
:107A5000D4050020BC040020100A0020A002002051
:107A600044010020140801402DE9F05FFE48FF4961
:107A7000DFF8FCB3007E0A1D131D0128584650D0C4
:107A800030F85A4F0C8041881180BBF85E00188096
:107A9000FDF792FEDFF8DC83F74C49F2CD32B8F9FE
:107AA0001E106183B8F9200043F6CC4701EB40007B
:107AB00050430014A083B4F92230B4F9205000FBE5
:107AC00003F201FB052242F38F326282B4F91660A1
:107AD00068437E4340F23337B6137A4306EBA23253
:107AE00001FB1300E54EE2828013E54DA082706C2D
:107AF0002860296928468847E2492889488008463D
:107B0000FDF73CFFE04F4FF0000A4FF001093878D5
:107B1000A4F1540508280CD0618E218204283ED09F
:107B20001AE030F8604F0C8041881180BBF8640087
:107B3000ADE7D64890F92B10491C02292DD890F8B2
:107B4000681019B1B4F85200208205E0618E2182DC
:107B5000A4F8521080F86890B4F91410B4F90A002F
:107B6000CB4AF9F78FFCE062BBF91611884204DDBD
:107B7000C748E162027A91400162287808B185F82D
:107B800000A0387804280ED0C14AB4F91610B4F910
:107B90000800243AF9F776FC08E0608ED4E7D8F8BC
:107BA00024000014E062B07AA8B1BA48BA4EA062CC
:107BB0003060E06A70603046FCF7E2F8B44F307C29
:107BC000383F01280AD0A06A3860B4480178C90754
:107BD00008D0406907E04FF4AF70E7E7706938609C
:107BE000B06900E0E06A7860A9483838FCF73CFAF0
:107BF000A14CA14934F8100F3C39FFF7A9FDA96940
:107C00006967B4F91010B868A846B4F9122000FBEF
:107C100001F5FB68504303FB125503FB010045F3DC
:107C20008F37A78640F38F36E6869D4C20466780C7
:107C3000A680FEF745FA904D207F383D01282FD0D1
:107C4000704241104DF6B350474369803A142A8080
:107C50004046A8F80A608B188381891AA8F80E108C
:107C60008BF80CA0B8F90A305C46002B01DD84F8D3
:107C70000C90B8F90C00002802DD217B891C2173CF
:107C8000B8F90E20002A02DD217B091D2173217B1A
:107C900007291CD2DFE801F01B1732142E1930001F
:107CA000B4F920304DF6B352584241106980B4F90E
:107CB0001E00504302142A804046A8F80A30CAE742
:107CC00084F80D9003E0022100E0032161736A490A
:107CD000744E754F09780129617B11D040F67E5AA8
:107CE00041F6FF2B07297BD2DFE801F07AFDFCFB90
:107CF000FAF9F8000421E9E70521E7E70621E5E7BD
:107D00000729F0D2DFE801F06C04234D6D97DA000B
:107D100001461846FBF7D0FE2860B5F90200B5F918
:107D2000001043F2046201445143090CA4F85A10B4
:107D30005043000CA4F85C00A4F85EA0002130467B
:107D4000F8F708FF00213846F8F704FF84E14042C5
:107D500001B2504200B2FBF7AFFE2860B5F9020055
:107D600043F204614143090CA4F85A10B5F900101C
:107D7000084443F204614843000CA4F85C00A4F8F2
:107D80005EA000213046F8F7E5FE00213846F8F7FE
:107D9000E1FEBDE13046F8F767FF01231A460721EF
:107DA000BAE019461046FBF787FE2860A4F85AA0EF
:107DB000B5F90200B5F9001043F2046201445143E1
:107DC000090CA4F85C105043000CA4F85E000021DC
:107DD0003046F8F7BFFE00213846F8F7BBFEEDE16C
:107DE000A5E05942404209B200B2FBF765FE2860A7
:107DF000A4F85AA0B5F9020043F204614143090C0A
:107E0000A4F85C10B5F90010084443F2046148433B
:107E1000000CA4F85E0000213046F8F79BFE00211C
:107E20003846F8F797FE21E23046F8F71DFF0123A8
:107E30001A46052170E01146FBF73EFE2860B5F9B1
:107E4000020043F204614143090CA4F85A10A4F85B
:107E50005CA0B5F90010084443F204614843000CEB
:107E6000A4F85E00002121E090090020342C01409C
:107E7000A00200202405002068000020440100200A
:107E800030040020F0030020F7060020240A002020
:107E900090080020A2FEFFFFE8090020080900204A
:107EA000C409002000240140002801403046F8F7B2
:107EB00051FE00213846F8F74DFE2DE2504201B246
:107EC000584200B2FBF7F8FD2860B5F90200B5F999
:107ED000001043F204620144514305E024E2C9E189
:107EE00070E119E1BDE063E0090CA4F85A105043B9
:107EF000A4F85CA0000CA4F85E0000213046F8F75E
:107F000029FE00213846F8F725FE63E23046F8F7EF
:107F1000ABFE01231A4606213846F8F7A5FE0121DB
:107F20003046F8F717FE01213846F8F713FEFC4DEE
:107F3000FC4E2889308068897080288AB08030465D
:107F4000F9F7CEFCB4F85A00F1880844A4F86000B0
:107F5000B4F85C0031890844A4F86200B4F85E000B
:107F600071890844A4F86400317EA5F13400012928
:107F700076D034F85A1F018061884180A1888180C1
:107F8000E74902882C390A8042884A8080888880A4
:107F9000E348896A2C38884795F8360000287DD058
:107FA000F9F760F815F8360F401E2870BDE8F09F0D
:107FB00001461846FBF780FD2860B5F9020040F63F
:107FC0008151484380136880B5F9001040F6815212
:107FD000514389134218A2F6815252425208298015
:107FE000A4F85E201044A4F85C00084424F85A0F5A
:107FF00000213046F8F7AEFD00213846F8F7AAFD1B
:1080000034F8021BA8F8021034F8022BA8F8042058
:1080100034F85E39A8F80630C1F5586083B2B3F57C
:10802000227F02D9A8F808A016E08A1A92B2404628
:10803000A8F81220B2EB430F01D96C390AE001F520
:10804000227189B20181B1F5586F05D380F8019092
:10805000ABEB0101A8F8081001231A46062199E6A6
:10806000BCE1404201B2504200B2FBF725FD28605E
:10807000B5F9020040F68151484381136980B5F992
:10808000000040F68152504380130A18A2F6815234
:10809000524228805208A4F85E2000E0A1E1114479
:1080A00024F85A1F0844608000213046F8F752FD3A
:1080B00000213846F8F74EFD34F8022BA8F80220CC
:1080C00034F8021BA8F8041034F85E39A8F806301A
:1080D000C1F5586083B2B3F5227F02D9A8F808A091
:1080E00016E08A1A92B24046A8F81220B2EB430F6B
:1080F00001D96C390AE001F5227189B20181B1F52B
:10810000586F05D380F80190ABEB0101A8F8081077
:1081100001231A4605213DE619461046FBF7CCFC23
:108120002860B5F9020040F6815148438013688009
:10813000B5F9001040F68152514389134218A2F656
:10814000815252422980520824F85A2F1044A080AC
:108150000844608000213046F8F7FCFC00213846D6
:10816000F8F7F8FC34F8021BA8F8021034F8021BE8
:10817000A8F80410C1F5586034F85E2983B2A8F855
:108180000620B3F5227F02D9A8F808A016E08A1AC3
:1081900092B24046A8F81220B2EB430F01D96C39D5
:1081A0000AE001F5227189B20181B1F5586F05D35A
:1081B00080F80190ABEB0101A8F8081001231A46E2
:1081C000072131E65942404209B200B2FBF774FC84
:1081D0002860B5F9020040F6815148438013688059
:1081E000B5F9001040F68152514389134218A2F6A6
:1081F000815252422980520824F85A2F104460803C
:108200000844A08000213046F8F7A4FC002138463D
:10821000F8F7A0FC34F8021BA8F8021034F8022B7F
:10822000A8F8042034F85E19A8F80610C1F55860C3
:1082300083B2B3F5227F02D9A8F808A016E08A1A03
:1082400092B24046A8F81220B2EB430F01D96C3924
:108250000AE001F5227189B20181B1F5586F05D3A9
:1082600080F80190ABEB0101A8F8081001231A4631
:108270000621D9E51146FBF71FFC2860B5F902007D
:1082800040F68151484381136980B5F9000040F6FA
:108290008152504380130A18A2F68152524252086A
:1082A00028801144A4F85C2024F85A1F0844A080B8
:1082B00000213046F8F74EFC00213846F8F74AFC1A
:1082C00034F8022BA8F8022034F8021BA8F8041096
:1082D00034F85E19A8F80610C1F5586083B2B3F5FA
:1082E000227F02D9A8F808A016E08A1A92B2404666
:1082F000A8F81220B2EB430F01D96C390AE001F55E
:10830000227189B20181B1F5586F05D380F80190CF
:10831000ABEB0101A8F8081001231A460521F5E589
:108320006800002090090020504201B2584200B27B
:10833000FBF7C2FB2860B5F9020040F681514843C3
:1083400080136880B5F9001040F6815251438913BB
:108350004218A2F68152524252082980A4F85C20A9
:108360001044A4F85E00084424F85A0F0021304657
:10837000F8F7F0FB00213846F8F7ECFB34F8020B75
:10838000A8F8020034F8022BA8F80420C0F55861C0
:1083900034F85E298BB2A8F80620B3F5227F02D903
:1083A000A8F808A016E0821A92B24146A8F8122056
:1083B000B2EB430F01D96C380AE000F5227080B2AD
:1083C0000881B0F5586F05D381F80190ABEB000040
:1083D000A8F8080001231A46072197E534F8601F22
:1083E000C9E505480088A0F5D04168393FF4DEAD05
:1083F000BDE8F05FF9F704BD182C01402DE9F0410C
:10840000904C9148B4F85A100288511A89B20F2939
:108410006FD30088A4F85A008C480088DFF83082B7
:10842000C0074FF000054FF0010741D0874AD4E95B
:108430000C1024321388B1EB530F02D21288511A58
:1084400008444FF4F371884200D208468149B1FBD9
:10845000F0F0616CC1F35101084406466064F7F71F
:10846000DEFF00227C4BF7F746FF4FF040427B4B8C
:10847000F7F741FF0E22F7F7ADFFF8F707F8A4F87A
:10848000A40094F86500401CC0B284F86500082878
:1084900034D36C4898F84620001F03789A4201D0E4
:1084A000027045806E4A13786E4A23B1458021E000
:1084B0006564A56458E0D8F89410A1F5FA618E427D
:1084C00011DD616D8B1C9E4205DDB0F902100A2999
:1084D0000DDA491C06E08E4205DAB0F902100029D7
:1084E00008DD491E4180B0F902000A2802DB17703E
:1084F00001E0A2E01570666584F865505A484FF4B3
:10850000A5420178C1F38101012949D002294AD04D
:1085100044F687712181A4F8A020B0F9243089B2F3
:108520004B439B13A4F89C30B0F90E00002370431A
:10853000B0FBF1F0A16CC0F3D100C1EBC101C902E5
:1085400000EB9130A064F017810341EA9641B0033B
:10855000F7F7EAFDB4F8A210C1EBC101C902C008E7
:1085600000EB9130A4F8A200616CA06E0844A066F4
:1085700094F86C20521CD2B284F86C20082A05D3DF
:10858000C008A4F86E0084F86C50A566374A384ECF
:10859000D388580633D498F80F00022806D02CE070
:1085A00043F20451B6E744F24621B3E7B06840F61F
:1085B0009916B04221DD94F8380094F88660B042F4
:1085C0000CD084F8860094F83D0000F00106C0F35A
:1085D0004000864202D1A4F8825004E0B4F8820040
:1085E000B0F5966F05D2B4F88200401CA4F8820062
:1085F00005E043F08000D08001E0A4F882501148EB
:1086000094F83F20B0300C2A01D2C57400E0C77442
:10861000174B41F2482641F2504C93F83C400C4B2A
:108620000C2AB3F882300AD3B14208DB012C06D001
:10863000614502DD002B00D18774BDE8F0818574AF
:10864000FBE7000044010020000700200004004078
:10865000A00200204564BD0100209C40133B334034
:10866000EE030020EF030020BC040020100A0020CD
:10867000240500202DE9F041384C394E394F20783F
:1086800041F23331C2074FF000050CD0A28962B32A
:1086900094F90700002800DA4042C0B2032829D22A
:1086A00040F2AE702AE0A570E5732F4AE571A5810E
:1086B00092F83830237220F00800A18040F00200C8
:1086C00020703D867560B560F560916C490005D0FD
:1086D00041F68461A18140F010002070C0B240F0EA
:1086E000010020706574BDE8F081658120F0100004
:1086F000207015E0042803D240F6510060810FE09D
:10870000052802D240F69910F8E740F6CC42062838
:1087100003D3072801D3082801D2628100E06181D8
:1087200097F89D0098B9B088102301B2B4F90A00F7
:108730003622FCF79BF87060F168401AB168084473
:10874000B060B6F900104843C013F0603886388E28
:1087500010B10120A070C6E7A570C4E7180C002076
:1087600080060020A0020020440100202DE9F041F5
:10877000554C2678F0077CD05448217A544D90F817
:10878000380081427BD0534A2346DFF84CC1575C06
:1087900093F90E2093F90730874203D01CF801703B
:1087A000874213D146F002065B1C26705BB2E37170
:1087B0001CF80110814201D15B1CE37194F9071090
:1087C000062901DD0621E171521C1CE0434F17F818
:1087D00001C0434F844503D017F801C0844513D12D
:1087E00026F002065B1E26705BB2E371795C814263
:1087F00001D15B1EE37194F907306FF005018B42E4
:1088000000DAE171521EA273207294F907108A1CDB
:10881000042A02D941F68462A2812C4A01291278E5
:108820000ADD2B4B56079B6802D543F0080301E095
:1088300023F00803AB606070B1F1FF3F09DA510724
:10884000A96802D521F0080101E041F00801A96002
:108850006070F9F76FFDA078012810D12148806879
:10886000A3280CDA94F90700022803DD0220E07146
:1088700005E01EE06FF00101884200DAE171A08995
:10888000002630B1401E0004000CA08101D1E67129
:10889000A673E87B04280CD0B5F93010512341228F
:1088A0000020FBF7E3FF2886002802D1E07B10B10F
:1088B000A670BDE8F0810C4806700C480670207860
:1088C00020F001002070F4E7180C00204401002083
:1088D000A0020020089500080E9500081A950008CF
:1088E000209500082405002014070020F70600202A
:1088F000B83ED93C223B8E391938BF367D355034CD
:1089000036332D3234314830692F962ECE2D0F2D2F
:108910005A2C000000361C070038AA0A003AAA0A9E
:10892000003CCC0C003ECC0C0040380E0042380E0F
:108930000044380E0046380E0048380E004AC71171
:10894000004CC711004EC7110050C7110052C7118B
:108950000054C7110056C7110058C711005AC7115B
:10896000005CC711005EC7110060C7110062C7112B
:108970000064C7110066C7110068C711006A0000D3
:108980000036000000388E03003A8E03003CFA04E3
:10899000003EFA0400401C0700421C0700441C076C
:1089A00000461C0700481C07004A8808004C88083D
:1089B000004E880800508808005288080054880833
:1089C0000056880800588808005A8808005C880803
:1089D000005E8808006088080062880800648808D3
:1089E0000066880800688808006A000000360000F9
:1089F00000388E03003A8E03003CFA04003EFA046D
:108A000000401C0700421C0700441C0700461C07CE
:108A100000481C07004A8808004C8808004E880857
:108A200000508808005288080054880800568808BA
:108A300000588808005A8808005C8808005E88088A
:108A4000006088080062880800648808006688085A
:108A500000688808006A0000003A2202003C8E0389
:108A6000003EB0050040D2070042AA0A0044CC0CE8
:108A70000046EE0E00481111004A3313004C9F14BB
:108A8000004E0B16005077170052771700547717D7
:108A90000056771700587717005A7717005C77173A
:108AA000005E77170060771700627717006477170A
:108AB0000066771700687717006A7717006C7717DA
:108AC000006E00000036000000388E03003A8E036E
:108AD000003CFA04003EFA0400401C0700421C0758
:108AE00000441C0700461C0700481C07004A880871
:108AF000004C8808004E88080050880800528808FA
:108B0000005488080056880800588808005A8808C9
:108B1000005C8808005E8808006088080062880899
:108B2000006488080066880800688808006A0000F9
:108B3000003A2202003C8E03003EB0050040D207FE
:108B40000042AA0A0044CC0C0046EE0E0048111167
:108B5000004A3313004C9F14004E0B160050771739
:108B600000524F1A0054BB1B0056271D0058931E7D
:108B7000005A0020005C6C21005ED8220060442472
:108B80000062B0250064662600661C2700681C276A
:108B9000006A1C27006C1C27006E000000340000D7
:108BA0000036000000380000003A0000003C0000E1
:108BB000003E0000004000000042000000440000B1
:108BC0000046000000480000004A0000004C000081
:108BD000004E000000500000005200000054000051
:108BE0000056000000580000005A0000005C000021
:108BF000005E0000006000000062000000640000F1
:108C000000660000006844145858587011115858F4
:108C10005870411158584870111448585870141120
:108C2000584858703D1A0056E11A0054E11A005293
:108C3000851B0050281C004ECC1C004C141E004A02
:108C4000B81E00485C1F004600200044A3200042DC
:108C5000EB2100403323003E7A24003C6626003A94
:108C6000AE270038F5280036E12A0034CC2C00323B
:108C7000142E00305C2F002EA330002CEB31002A84
:108C8000333300287A340026C23500240A37002204
:108C900051380020E13A001E283C001CB83E001A62
:108CA0000040001800400016004000140040001270
:108CB000004000100040000E0040000C0040000A80
:108CC0000040000800400006004000040040000290
:108CD0000040000001020304050005000102030436
:108CE0000104000305020000F0010000360100004D
:108CF000F8000000BA0000007C0000007C000000CA
:108D00007C00000041141411111444111414411179
:108D10000000290052007B00A400CC00F5001E01D9
:108D2000470170019901C201EA0113023C02650288
:108D30008E02B602DF020803300359038203AA033E
:108D4000D303FB0324044C0475049D04C504EE0402
:108D500016053E0567058F05B705DF0507062F06D3
:108D600057067F06A706CE06F6061E0746076D07BE
:108D70009507BC07E4070B08320859088108A808C2
:108D8000CF08F6081D0944096A099109B809DE09E6
:108D9000050A2B0A520A780A9E0AC40AEA0A100B2C
:108DA000360B5C0B820BA80BCD0BF30B180C3E0C97
:108DB000630C880CAD0CD20CF70C1C0D410D650D2D
:108DC0008A0DAF0DD30DF70D1C0E400E640E880EEC
:108DD000AC0ECF0EF30E170F3A0F5E0F810FA40FDC
:108DE000C70FEA0F0D103010531075109810BA10FD
:108DF000DD10FF102111431165118711A911CA114E
:108E0000EC110D122E12501271129212B312D412D2
:108E1000F41215133613561376139613B713D7138C
:108E2000F61316143614561475149414B414D3147B
:108E3000F214111530154E156D158C15AA15C8159F
:108E4000E7150516231641165F167C169A16B716F7
:108E5000D516F2160F172C17491766178317A01788
:108E6000BC17D917F51711182E184A18661881184B
:108E70009D18B918D418F0180B19261942195D1944
:108E800078199219AD19C819E219FD19171A311A72
:108E90004C1A661A801A991AB31ACD1AE61A001BD0
:108EA000191B331B4C1B651B7E1B971BAF1BC81B61
:108EB000E11BF91B121C2A1C421C5A1C721C8A1C26
:108EC000A21CBA1CD21CE91C011D181D301D471D17
:108ED0005E1D751D8C1DA31DBA1DD01DE71DFD1D3A
:108EE000141E2A1E401E571E6D1E831E981EAE1E87
:108EF000C41EDA1EEF1E051F1A1F2F1F451F5A1F03
:108F00006F1F841F991FAE1FC21FD71FEC1F0020A9
:108F100000006400C9002D019201F7015B02C0024C
:108F200024038903ED035204B6041A057F05E30503
:108F30004706AB060F077307D7073B089F080209D0
:108F40006609C9092D0A900AF30A560BB90B1C0CC5
:108F50007F0CE20C440DA60D090E6B0ECD0E2F0FEB
:108F6000900FF20F5310B41015117611D71138125B
:108F70009812F8125813B81318147714D61435151C
:108F80009415F3155116B0160E176B17C91726183E
:108F90008318E0183D199919F519511AAD1A081BD3
:108FA000631BBE1B181C731CCD1C261D801DD91DE8
:108FB000321E8A1EE31E3B1F921FEA1F412098208B
:108FC000EE2044219A21EF2145229922EE224223CC
:108FD0009623E9233C248F24E22434258525D725B4
:108FE00028267826C82618276827B7270628542851
:108FF000A228EF283D298929D629222A6D2AB82AB4
:10900000032B4D2B972BE12B2A2C722CBB2C022DE2
:109010004A2D912DD72D1D2E632EA82EEC2E302FEC
:10902000742FB82FFA2F3D307F30C03001314131DD
:109030008131C13100323F327D32BA32F7323433BE
:109040007033AC33E73322345C349534CE34073597
:109050003F357735AE35E4351A3650368536B93674
:10906000ED36203753378637B737E937193849385F
:109070007938A838D738053932395F398B39B7395B
:10908000E2390D3A373A603A893AB23ADA3A013B74
:10909000283B4E3B733B983BBD3BE03B043C263CAE
:1090A000483C6A3C8B3CAB3CCB3CEA3C093D273D11
:1090B000443D613D7D3D993DB43DCE3DE83D013EA1
:1090C0001A3E323E493E603E763E8C3EA13EB53E63
:1090D000C93EDC3EEF3E013F123F233F333F433F5B
:1090E000513F603F6E3F7B3F873F933F9E3FA93F8D
:1090F000B33FBC3FC53FCD3FD53FDC3FE23FE83FFC
:10910000ED3FF13FF53FF93FFB3FFD3FFF3FFF3FA5
:10911000FF3F0000E7382C35002020EF20372023C8
:1091200033202620210000800200040008001000E7
:1091300000020004000804000002000400080010FF
:10914000002000400080040000000080000000407B
:1091500000000020000000100000000800000004D3
:10916000000000020000000100008000000040003C
:1091700000002000000010000000080000000400B3
:109180000000020000000100008000000008014013
:10919000000C0140000C0140000C0140000C01409B
:1091A000000C0140000C0140000C01400010014087
:1091B000001001400010014000100140001001406B
:1091C0000010014000100140001001400014014057
:1091D00004080140040C0140040C0140040C01404F
:1091E000040C0140040C0140040C0140040C01403B
:1091F000041001400410014004100140041001401B
:10920000041001400410014004100140041001400A
:109210000414014008080140080C0140080C0140FA
:10922000080C0140080C0140080C0140080C0140EA
:10923000080C0140081001400810014008100140CE
:1092400008100140081001400810014008100140BA
:1092500008100140081401400C0801400C0C0140AA
:109260000C0C01400C0C01400C0C01400C0C01409A
:109270000C0C01400C0C01400C1001400C10014082
:109280000C1001400C1001400C1001400C1001406A
:109290000C1001400C1001400C140140100801405A
:1092A000100C0140100C0140100C0140100C01404A
:1092B000100C0140100C0140100C01401010014036
:1092C000101001401010014010100140101001401A
:1092D0001010014010100140101001401014014006
:1092E000000000000000000000000000000000007E
:1092F0000000000014080140140C0140140C01404F
:10930000140C0140140C0140140C0140140C0140D9
:10931000140C0140141001401410014014100140BD
:1093200014100140141001401410014014100140A9
:10933000141001401414014000000000000000005F
:10934000000000000000000000000000FFFFFF0F11
:109350000FFFFFFFFFF0FFFFFF0FFFFFFFFFF0FF1B
:109360000FFFFFFFFFF0FFFFFF0FFFFFFFF0FFFF0B
:109370000FFFFFFFFFF0FFFFFF0FFFFFFFFFF0FFFB
:10938000FFFF0FFFFFFFFFF0FFFFFF0FFFF0FFFFEB
:109390000000004040000000000400000040000009
:1093A0000000040040000000000400000040000035
:1093B0000004000040000000000400000040000025
:1093C0000000040000004000000000040000004015
:1093D0000004000000000080800000000008000081
:1093E000008000000000080080000000000800006D
:1093F000008000000008000080000000000800005D
:10940000008000000000080000008000000000084C
:109410000000008000080000000000202000000084
:1094200000020000002000000000020020000000F8
:1094300000020000002000000002000020000000E8
:1094400000020000002000000000020000002000D8
:109450000000000200000020000200000000006088
:109460006000000000060000006000000000060030
:109470006000000000060000006000000006000020
:109480006000000000060000006000000000060010
:109490000000600000000006000000600006000000
:1094A0000080020004000800100000020004000810
:1094B00004000002000400080010002000400080AA
:1094C00004000000FF7FFFFFFDFFFFFFFBFFFFFF2A
:1094D000F7FFFFFFEFFFFFFFFFFDFFFFFFFBFFFFBA
:1094E000FFF7FFFFFBFFFFFFFFFDFFFFFFFBFFFF9E
:1094F000FFF7FFFFFFEFFFFFFFDFFFFFFFBFFFFFF4
:10950000FF7FFFFFFBFFFFFF0102030405000203D3
:109510000405000103040500010205000102030423
:1095200004050001020355050010AA1A5525003054
:10953000AA3A0000AA0A55150020AA2A5535FF3F6D
:10954000609500080000002028070000E8060008D9
:109550005496000828070020B00900009463000812
:1095600045020406082D0102030404054C06070801
:109570000913792B1B088D04211355152A40061950
:1095800008019713C53D1B08E9041AE504012D17CE
:10959000020604050103148020FF8BAA0A02019C25
:1095A00015AA0A551500085920AA2A5535FF3F0764
:1095B0002903010504060203127C1573FFFF04FF53
:1095C0008080010125025B6402130A1301671208FF
:1095D0001201100C0504060203010103070505280A
:1095E0000B010203040206070303040C3D070604F3
:1095F0000509191F191904310506062FAA1A381E64
:10960000AA1A064902290C2902312E40FD39692681
:109610000211042F405F020C26405B262ACD55150F
:109620005515123902017F0316D0071AFF01013BBD
:109630000261AA6C080108A80916C491220312103D
:109640000A17401C12600A16901B01491315670285
:04965000000800000E
:020000040800F2
:10FC00004A46545A594D46312D4E3330202020203B
:10FC1000050406020301AA0AAA0AAA0AAA0AAA0A4B
:10FC2000AA0ADE3F00100000FF0131000201664613
:10FC300000400040513800400040004000400101B9
:10FC400000400040FF387B257B257B25FF003333B8
:10FC50000201401F00016626B81E6626FFFFFFFF57
:10FC6000FFFF01010100010000000300000202008B
:04FC70000000AA5591
:04000005080000ED02
:00000001FF
